:020000040800F2
:2000000040100020D5000008A9250008E31F000800000000000000000000000000000000B3
:20002000000000000000000000000000312700080000000000000000252600085529000887
:20004000E7000008E7000008E7000008E7000008E70000087D030008E7000008E70000088F
:2000600000000000E700000865030008E7000008E70000082D23000800000000E7000008FC
:2000800000000000E70000080000000000000000E700000800000000E7000008E7000008A4
:2000A000E7000008E7000008E700000881300008E7000008E70000080000000000000000DC
:2000C0000348854600F0A0F80048004735340008401000200448804704480047FEE7FEE7A2
:2000E000FEE7FEE7FEE7FEE7152A0008C100000830B50B46014600202022012409E00D461C
:20010000D5409D4205D31D469540491B2546954040191546521E002DF1DC30BDF0B51FB4B4
:200120000646002082B005464024019100901BE0019922460F46304600F054F8049A059B0E
:20014000801A994110D310461946224600F03AF8361A8F410197224601200021009F00F018
:2001600031F838184D4100902046641E0028DFDC019B00982946324607B0F0BD03460B4307
:200180009B0703D009E008C9121F08C0042AFAD203E00B780370401C491C521EF9D27047B1
:2001A000D2B201E00270401C491EFBD270470022F6E710B513460A4604461946FFF7F0FF26
:2001C000204610BD10B5202A04DB0146203A9140002010BD914020239C1A0346E34019430D
:2001E000904010BD10B5202A04DB0846203AD040002110BD0B46D340D0402024A21A914089
:200200000843194610BD0000064C0125064E05E0E36807CC2B430C3C98471034B442F7D3FF
:20022000FFF752FF0C3500082C350008F0B505460E460024AF1905E029786D1CA0B202F042
:200240003BFF0446BD42F7D3A0B2002102F034FF04462046002102F02FFF04462046F0BD6B
:2002600010B504210EE002785200037880242340002B01D01B2300E000235A400270401CB3
:200280004A1ED1B20029EEDC10BD30B502460B460021012000BF505419544C1CE1B24400E4
:2002A00080250540002D01D01B2500E000256C404440E0B20128EED11578FF24A55430BDD1
:2002C00070B50246002000BF002808DD0F4D2D682D5CFF26751B0E4E3668715D00E00021CD
:2002E00063254D402C46042308E04D00CE113543E9B225464D402C465D1EEBB2002BF4DCAC
:200300001454451CEDB2281EDED170BD040000200000002010B502460B460020002100BFB1
:2003200000BF545C844201D11954FF214C1CE4B2211EF6D1441CE4B2201EF1D110BD00BFA3
:200340000B780370401C491C531EDBB21A1EF7D1704701784278027082784270C2788270B4
:20036000C170704710B5034800F090F9024800F08DF910BDDC0900209409002010B50121D6
:200380008902034800F04CF9022000F01DFB10BD0004005070470000FFB581B004460E46CD
:2003A0001746002500F0C8FA00BF29E01948006881000498814207D300201649086000F0E7
:2003C00083FA002005B0F0BDA80032582168022000F08AFA00280BD120680068A900715867
:2003E000884201D00220EDE72068001D206001E00120E7E76D1C07480068401C0549086025
:20040000BD4203D2206804498842CFD900F05CFA0020D7E720000020FBFB000800210A4AEA
:2004200051610A494968012252021143074A51601146496808221143044A51600021C209C8
:20044000D201116070470000240A0020002002407FB504460D460020039000F06DFA0020F6
:2004600000900194E809029003A9684600F0E6F9002804D000F028FA002004B070BD00F0AC
:2004800023FA0120F9E70000002039498969FF2201321140914208D13649496902221143B0
:2004A000344A5161FF210131084331498969012252021140914208D12E49496901221143EF
:2004C0002C4A516101214902084329498969012292021140914208D1264949690822114385
:2004E000244A5161012189020843214989690122D2021140914208D11E4949690422114301
:200500001C4A51610121C902084319498969012252031140914208D116494969102211432B
:20052000144A516101214903084311498969012252041140914207D10E4949692022114392
:200540000C4A51612021084309498969012212041140914208D10749496940221143054A86
:200560005161012109040843014988617047000000200240240A002070B5044600F034FB27
:2005800005460BE0601C002808D0002C04D000F02BFB401BA04201D9032070BD1F488069DC
:2005A000C007C00F0028EDD11C48806902210840022801D11949886118488069FF21013125
:2005C0000840884223D0154880694900084088421DD01248806949000840884217D00F48AC
:2005E000806949000840884211D00C4880698900084088420BD009488069090108408842CD
:2006000005D00648806949100840884203D1FFF73BFF0120C1E70020BFE70000002002406E
:2006200070B504460D462946204600F0D3FA70BD70B5044600252520005D022803D00420E2
:20064000E063012520E0206800680E218843216808602068006840084000216808601C21B0
:20066000606C084001218140206C416001212520015500BF00212420015500BFA06B00282D
:2006800002D02046A16B8847284670BD70B50446206C0568206806681C20616C01400420E0
:2006A0008840284000281DD004203040002819D02068006820210840002805D120680068E9
:2006C00004218843216808601C21606C084004218140206C4160206B00285AD02046216B06
:2006E000884756E01C20616C0140022088402840002825D002203040002821D020680068A1
:2007000020210840002808D1206800680A218843216808600121252001551C21606C08406A
:2007200002218140206C416000BF00212420015500BFE06A00282CD02046E16A884728E079
:200740001C20616C0140082088402840002820D00820304000281CD0206800680E21884349
:20076000216808601C21606C084001218140206C41600120E06301212520015500BF002126
:200780002420015500BF606B002802D02046616B884770BD70B50446002C01D1012070BD52
:2007A000244A2168881A1421FFF7A2FC8000606420480838206402212520015520680568B4
:2007C0001D480540E168A06808432169084361690843A1690843E1690843216A08430543E1
:2007E0002068056001218903A068884217D011487830806A1C22616C11400F228A40904390
:200800000C49783188621C22616C11406068884008497831896A08430649783188620020CA
:20082000E0630121252001550021242001550020B5E70000080002400F80FFFFF8B5044673
:200840000E460127002500BF1C48007C012801D10220F8BD01201949087400BF1848FFF772
:200860008BFE0746002F22D1401E3060656817E02846FFF7D3FD1248FFF77EFE0746114828
:200880004068082188430F49486008464068491588430C494860002F01D0356006E0803570
:2008A000A068C00161684018A842E1D800BF00BF00200249087400BF3846CAE7240A00200A
:2008C00050C3000000200240064840680221084304494860084640680121084301494860F5
:2008E0000020704700200240F8B507460C461546012600BF0E48007C012801D10220F8BD8E
:2009000001200B49087400BF0A48FFF735FE0646002E06D10649486125600648FFF72CFE70
:20092000064600BF00200249087400BF3046E6E7240A002050C300001D484068C007C00FBF
:20094000002816D000BFEFF31080014600BF72B61848174AD0601848D06000BF81F31088DE
:2009600000BF10464068C007C00F002801D0012070470F48406802221040022815D100BF11
:20098000EFF31080014672B60C48094A10610C481061084680F3108800BF1046406802225F
:2009A0001040022801D10120E2E70020E0E7000000200240EFCDAB8905040302BFAE9D8C24
:2009C000161514137047000010B50446054840692040002804D0034844612046FFF7F2FF70
:2009E00010BD00000004014070B50346002200240020DAE0012696400D6835402C46002CD2
:200A000077D04D68022D02D04D68122D15D1D508AE001D462035A8595507EE0E0F25B5403A
:200A20000646AE4330465607F60E0D69B5402843D508AD001E46203670514D68012D08D00C
:200A40004D68022D05D04D68112D02D04D68122D18D1986856000325B5400646AE43304615
:200A60005600CD68B540284398605868012595400646AE43304610264D6835402D099540BA
:200A800028435860186856000325B5400646AE4330460D79AD07AD0F5600B5402843186069
:200AA000D86856000325B5400646AE43304656008D68B5402843D860012636074D6835405F
:200AC000B54271D13C4D6D6B012635433A4E75633A4D9608B600A85995072E0F0F25B5409F
:200AE0000646AE43304605252D07AB4202D1002515E059E0324DAB4201D101250FE0314D01
:200B0000AB4201D102250AE02F4DAB4201D1032505E02E4DAB4201D1052500E006259607B1
:200B2000360FB5402843254D9608B600A851284D28680546A5432846012636044D68354020
:200B4000B54202D1054625432846214D286068680546A5432846012676044D683540B54281
:200B600002D1054625432846194D6860A8680546A5432846012636054D683540B54202D14C
:200B8000054625432846124DA860E8680546A5432846012676054D683540B54202D10546FB
:200BA000254328460A4DE860521C0D68D540002D00D01FE770BD00000010024008000140FD
:200BC0000004005000080050000C0050001C00500004014042694A4042617047002A01D0D2
:200BE000816100E08162704701480068704700002800002002480068401C01490860704772
:200C00002800002010B50024084800684021084306490860002000F00BF8002801D0012457
:200C200001E000F0FDF8204610BD00000020024070B5044600257D21C90009480068FFF7AF
:200C400057FA064600F0DAFE002801D0012504E000222146501E00F0FFF8284670BD0000B3
:200C60002C0000207047704710B5044622480078401C2149087008460078030002F068FB6D
:200C80000A3A060C12181E252C31363A012109031A48FFF7C5FC2DE0012109031748FFF7ED
:200CA000BFFC27E0012149031448FFF7B9FC21E0012149031148FFF7B3FC1BE00121C903A7
:200CC00005200007FFF7ACFC14E00121C90305200007FFF7A5FC0DE008210848FFF7A0FCAD
:200CE00008E008210548FFF79BFC03E000200249087000BF00BF10BD240000200004005060
:200D000070477047704710B5044620680068C007C00F01214840484000280CD02068806873
:200D2000084048404840002805D00120216848602046FFF799FF2068006802210840400875
:200D400000280BD02068806808404008002805D00220216848602046FFF784FF2068006871
:200D600004210840800800280BD02068806808408008002805D0042021684860204600F093
:200D80004DF82068006808210840C00800280BD0206880680840C008002805D008202168B4
:200DA00048602046FFF7ACFF2068006810210840000900280BD02068806808400009002826
:200DC00005D01020216848602046FFF74CFF2068006820210840400900280BD02068806801
:200DE00008404009002805D02020216848602046FFF788FF206800684021084080090028C7
:200E00000BD02068806808408009002805D04020216848602046FFF774FF10BD70470000D5
:200E20000648406B01210843044948630846806B0904084301498863704700000010024085
:200E400000BFC206D20E01219140024A116000BF7047000000E100E070B504460D46164626
:200E60002946204601F0A2FB70BD000003480068FF21013108430149086070470070004079
:200E8000F8B5044620212068084020287CD120680840202800D100BF00278148806B012110
:200EA00009070840002805D17D48806B08437C49886301277B480068FF210131084000281C
:200EC00016D178480068084376490860FFF78CFE064606E0FFF788FE801B642801D903203F
:200EE000F8BD70480068FF21013108400028F1D06B480568032109050D4060680840A84201
:200F00000DD0091160680840884208D164480068012149040840884201D10120E0E7604830
:200F2000403000690321090408400546002D3DD060680840A84239D020212068084020287E
:200F400034D157484030006903210904884305465348403000690121C90408435049403115
:200F60000861084600690121C90488434C494031086108460561801528408915884215D129
:200F8000FFF732FE064608E039E0FFF72DFE801B4549884201D90320A2E7414840300069E2
:200FA000012149020840400A0028EED000BF00BF032109046068084088420AD13848006800
:200FC00009018843032212056168114008433449086000BF324840300069032212046168A0
:200FE000114008432E494031086100BF012F05D12B48806B890588432949886300BF2078D4
:20100000C007C00F002809D025484030C06880088000A168084322494031C8600221206829
:201020000840022809D11E484030C0680C218843E16808431A494031C860042120680840E9
:2010400004280AD116484030C0680321890288432169084312494031C86008212068084057
:2010600008280AD10E484030C068032109038843616908430A494031C8608021206808400A
:2010800080280AD106484030C068032189048843A169084302494031C860002020E700000B
:2010A000001002400070004088130000F8B504460D46002C01D10120F8BD79480068C00785
:2010C000C00FA8420ED2764800684008400028437349086008460068C007C00FA84201D033
:2010E0000120E9E7022120680840022807D16D48C068F0218843A16808436A49C86020788A
:20110000C007C00F00284CD06068022809D165480068012149040840400C002824D10120D3
:20112000CAE76068032809D15E480068012149060840400E002817D10120BDE76068012856
:2011400008D15848006804210840800800280BD10120B1E753480068012149020840400AFA
:20116000002801D10120A7E74E48C06880088000616808434B49C860FFF736FD06466068F3
:2011800002280FD107E0FFF72FFD801B4649884201D9032090E74348C0680C21084008287C
:2011A000F1D134E0606803280FD107E0FFF71CFD801B3D49884201D903207DE73948C0689B
:2011C0000C2108400C28F1D121E0606801280FD107E0FFF709FD801B3349884201D9032011
:2011E0006AE73048C0680C2108400428F1D10EE007E0FFF7F9FC801B2B49884201D9032005
:201200005AE72848C0680C2108400028F1D124480068C007C00FA8420ED921480068400842
:20122000400028431E49086008460068C007C00FA84201D001203FE70421206808400428C5
:2012400008D11848C068072109028843E16808431449C860082120680840082809D11148BA
:20126000C0680721C90288432169C90008430D49C86000F049F80B49C968F0221140090941
:201280000A4A515CC8400A4908600020FFF7D0FC0746002F01D038460EE700200CE70000D5
:2012A000002002400010024088130000943400082C00002001480068704700002C0000200F
:2012C00000B5FFF7F7FF0549C968072212021140090A034A515CC84000BD0000001002403C
:2012E000A434000800B5FFF7E5FF0549C9680722D2021140C90A034A515CC84000BD000020
:2013000000100240A4340008FEB52E48C7680C203840002845D0042804D008280CD00C2822
:201320003ED10BE02748006810210840002801D0254C00E0254C41E0254C3FE00F20800444
:201340003840800C23490E5C032080053840800D401C01901B48C0680121090408400028EF
:2013600007D01B49714308460199FEF7C1FE054614E01448006810210840002807D012490C
:20138000714308460199FEF7B3FE054606E00F49714308460199FEF7ABFE05462C460DE09E
:2013A00000BF08484068072149030840400B00900098401C01218140CC0300BF00BF204655
:2013C000FEBD00000010024000093D000024F40000127A00AC340008FEB50446002C01D133
:2013E0000120FEBDF848C6680C210E40C768012109040F402078C007C00F002872D0082EAD
:2014000004D00C2E0FD1084687420CD1EE480068012149040840400C002863D060680028FE
:2014200060D10120DDE700BF012109046068884205D1E54800680843E349086027E005219F
:201440000904606888420ED1DF480068012189040843DD49086008460068012109040843C7
:20146000D949086013E0D8480068012109048843D54908600846006801210904084000902A
:2014800000BFD148006889008843CF49086000BF6068002813D0FFF7A7FB054606E0FFF7E7
:2014A000A3FB401B642801D903209AE7C6480068012149040840400C0028F0D012E0FFF7E0
:2014C00093FB054606E0FFF78FFB401B642801D9032086E7BC480068012149040840400C0D
:2014E0000028F0D102212068084002287AD1E0680290042E03D00C2E34D1002F32D1B24851
:201500000068042108408008002804D00298002801D1012065E7AC4840681F2109028843BF
:20152000216909020843A8494860084600680921884302990843A4490860FFF7E5FEA24988
:20154000C968F02211400909A04A515CC840A04908600020FFF76CFB01900198002841D015
:2015600001983EE70298002824D097480068092188430299084394490860FFF735FB05461F
:2015800006E0FFF731FB401B022801D9032028E78D4800680421084080080028F1D08A48C5
:2015A00040681F21090288432169090208438649486017E084480068400840008249086030
:2015C000FFF712FB054606E0FFF70EFB401B022801D9032005E77C48006804210840800849
:2015E0000028F1D1102120680840102867D1002E36D17548006849010840400A002804D05E
:20160000A069002801D10120EBE66F484068072149038843216A08436B494860084640680F
:201620000002000A217F0906084367494860206A400B401C01218140C8036349C968F0227E
:2016400011400909614A515CC840614908600020FFF7EEFA0190019800284BD00198C0E60B
:20166000A06900282CD058480068FF210131084355490860FFF7B8FA054606E0FFF7B4FA15
:20168000401B022801D90320ABE64F480068012149020840400A0028F0D04B4840680721EE
:2016A00049038843216A084347494860084640680002000A217F090608434349486019E0DC
:2016C00041480068FF21013188433F490860FFF78BFA054606E0FFF787FA401B022801D98A
:2016E00003207EE638480068012149020840400A0028F0D1082120680840082839D1606997
:2017000000281BD0304840300069012108432E4940310861FFF768FA054606E0FFF764FACA
:20172000401B022801D903205BE62748403000690221084040080028F0D01AE0224840302F
:20174000006940084000204940310861FFF74CFA054606E0FFF748FA401B022801D903202E
:201760003FE61948403000690221084040080028F0D1042120680840042879D10020009053
:201780001148806B89060840002806D10E48806B08430D498863012000900E480068FF21D3
:2017A0000131084000281ED10A480068084309490860FFF719FA05460EE0FFF715FA401B37
:2017C000642809D903200CE600100240943400082C0000200070004085480068FF210131E1
:2017E00008400028E9D000BFFF210131A068884205D18048006908437E49086130E0A06843
:2018000000280DD17B480069FF2101318843794908610846006909158843764908611FE087
:2018200005210902A06888420DD1724800690121890208436F4908610846006989150843EB
:201840006C4908610CE06B480069FF21013188436849086108460069091588436549086174
:2018600000BFA068002815D0FFF7BEF9054608E031E0FFF7B9F9401B5F49884201D9032031
:20188000AFE55C480069012149020840400A0028EFD013E0FFF7A8F9054607E0FFF7A4F972
:2018A000401B5549884201D903209AE551480069012149020840400A0028EFD1009801283F
:2018C00008D14C484038806B01210907884349494039886300BF606A00284CD00C2E69D005
:2018E000606A022848D1434840380068012109068843404940390860FFF776F9054606E074
:20190000FFF772F9401B022801D9032069E5394840380068012149060840400E0028EFD146
:20192000E16AA06A0843216B084332494039C968FD221204914308432E494039C860084651
:2019400000680121090608432A4940390860FFF74BF9054606E0FFF747F9401B022801D94F
:2019600003203EE5234840380068012149060840400E0028EFD038E01E4840380068012168
:20198000090688431B4940390860FFF72DF9054606E0FFF729F9401B022801D9032020E53C
:2019A000144840380068012149060840400E0028EFD11AE0606A012800D112E50D4840387A
:2019C000C768012000043840A16A88420BD10F2080043840E16A884205D103208005384054
:2019E000216B884201D00120FBE40020F9E4000000700040401002408813000070B5044677
:201A00002546681E0949884201D901200CE0681E074948610321081F00F0C8FD00200449E6
:201A2000886107200861002070BD0000FFFFFF0000E000E070477047FEB504462068C56902
:201A400020680668206887682807000F0190019800280ED12020284000280AD02020304050
:201A6000002806D0206E002802D02046216E8847FEBD019800287DD0F807C00F002804D188
:201A8000FF20213030400028F5D0E807C00F00280BD0FF2001303040002806D00120216850
:201AA0000862E06F01210843E0670220284000280AD0F807C00F002806D00220216808624C
:201AC000E06F04210843E0670420284000280AD0F807C00F002806D0042021680862E06F40
:201AE00002210843E0670820284000280ED020203040002803D1F807C00F002806D00820FB
:201B000021680862E06F08210843E067E06F002846D020202840002809D0202030400028BA
:201B200005D0206E002802D02046216E8847E06F00902068806840210840402804D0082127
:201B400000980840002826D0204601F053F82068806840210840402819D12068806888433F
:201B600021688860E06E00280DD02548E16E8863E06E00E015E0FEF75BFD002810D0E06E34
:201B8000816B88470CE02046FFF755FF08E02046FFF751FF04E02046FFF74DFF0020E06767
:201BA00066E701200005284000280CD0012080053840002807D001200005216808622046AA
:201BC000FFF738FF54E78020284000280AD080203040002806D0606E002802D02046616E88
:201BE000884745E740202840002807D040203040002803D0204601F00FF839E700BF37E7FD
:201C0000DD2B000810B50446002C01D1012010BDA069002800D000E000BF606F002805D14C
:201C2000002170200155204600F02CF824206067206800684008400021680860204600F059
:201C4000FBFF012800D1E2E7606A002802D0204600F014FF206840680921C9028843216821
:201C60004860206880682A21884321688860206800680121084321680860204600F076FFAC
:201C8000C5E7000010B586B00446142101A8FEF78EFA36492068884266D13548406B0121A6
:201CA000890308433249486300BF0846C06A012108432F49C8620846C06AC007C00F009043
:201CC00000BF00BF0320400201900220029000200390032004900420059001A905200007E3
:201CE000FEF782FE23482449086003204860002121488160C1608021016100214161816130
:201D00002021C16100210162FEF744FD002801D0FEF740FB00BF1848E066846200BF154816
:201D2000143816490860032048601021134881600021C16080210161002141618161C1614C
:201D40000162FEF727FD002801D0FEF723FB00BF0A48A066846200BF002201211B20FFF7CA
:201D60007BF81B20FFF76CF806B010BD00380140001002403000024094090020DC090020D9
:201D8000FFB585B004460D461746A06F20286FD1002D01D0002F02D1012009B0F0BD012120
:201DA0000903A068884208D12069002805D1E807C00F002801D00120EFE700BF7020005D8B
:201DC000012801D10220E8E701217020015500BF0020E0672220A067FEF706FF029058209C
:201DE00007535A20075300BF01210903A06888420AD12069002803D138495C20015324E041
:201E0000FF215C20015320E0A06800280AD12069002803D1FF215C20015316E07F215C2040
:201E2000015312E001210907A06888420AD12069002803D17F215C20015306E03F215C20C6
:201E4000015302E000215C20015300BF5C20005B039001210903A068884205D120690028AB
:201E600002D10026049502E02E460020049025E031E008980090002220212046029B01F029
:201E8000C9F8002801D0032087E7002E09D12068406A03990840049908800498801C0490E8
:201EA00006E02068406A0399C9B208403070761C5A20005B401E81B25A2001535A20005B70
:201EC0000028D6D12020A06700BF00217020015500BF002061E702205FE70000FF01000097
:201EE000FFB583B004460D461746606F202875D1002D01D0002F02D1012007B0F0BD0121FD
:201F00000903A068884208D12069002805D1E807C00F002801D00120EFE700BF7020005D29
:201F2000012801D10220E8E701217020015500BF0020E06721206067FEF756FE0190502035
:201F400007535220075301210903A068884205D12069002802D10026029502E02E460020CE
:201F6000029021E006980090002280212046019B01F050F8002801D00320BEE7002E09D1D9
:201F800002980088C005C00D216888620298801C029003E0307821688862761C5220005BF5
:201FA000401E81B2522001535220005B0028D9D106980090002240212046019B01F02AF865
:201FC000002801D0032098E72020606700BF00217020015500BF00208FE7FFE702208CE7C9
:201FE000704700BFFEE7000070B5044608492068084001214907884207D16568206880F31A
:20200000088800BFA847012070BD0020FCE700000000FE2FFEB504460D461948019000279B
:2020200000200090002628E028460199FEF760F83030C2B238467F1C225428460199FEF70D
:2020400057F80D460A210198FEF752F80190781E205C302801D1012000E00020009900292B
:2020600001D1012100E000210840002801D0002702E00098401C0090761C0A2ED4D3FEBD71
:2020800000CA9A3BF8B505460C460D200090E03410222146284601F02FF8103C00BF2846EE
:2020A00000F0B2F810222146284600F0C7F8103C0426002706E0E81900F015F8701EC6B249
:2020C000381DC7B2002EF6DC0098401EC0B200900028E4D1284600F097F810222146284669
:2020E00000F0ACF8F8BD18B504466078A1784840E1784840694608702078A1784840E1786D
:20210000414068464170207861784840E178414068468170207861784840A178414068462C
:20212000C1702046FEF79CF8207861784840694609784840694608706078A178484069467F
:202140004978484069464870A078E1784840694689784840694688702078E17848406946CF
:20216000C97848406946C8702046FEF779F82078A1784840694609784840694608706078F3
:20218000E1784840694649784840694648702078A17848406946897848406946887060780F
:2021A000E17848406946C97848406946C8702046FEF756F86078A1784840E1784840217843
:2021C000484020706946087821784840694608704878217848406946487088782178484007
:2021E000694688706846C178207841406846C1700078207068464078607068468078A07065
:202200006846C078E07018BD417B427A4273427942724278427141708178827A827081721F
:202220008179827B82718173C178C279C270C27AC271C27BC272C1737047000010B500BFCB
:202240000378064CE35C0C7863400370401C491C531EDBB21A1EF3D110BD000030010020FF
:202260007CB504462FA0006800902F4E202500BF30782070641C761C681EC0B2051EF7D16E
:20228000211F042201A8FEF75AF8202547E02846E917C90E091849114901691A1AD101A85B
:2022A000FEF757F8042101A800F046FB0422694601A800F021FF69460878400009788022BB
:2022C0001140002901D01B2100E000214840694608700CE02846E917C90E091849114901D1
:2022E000691A102903D1042101A800F025FB21462039042201A800F0FFFE6846007920703D
:20230000641C684640792070641C684680792070641C6846C0792070641C281DC5B2F02D3F
:20232000B5DB7CBD010000007434000810B50248FEF7E9FC10BD00008C08002008B500BF3D
:202340000648006B01210843044908630846006BC007C00F009000BF00BF08BD001002402B
:2023600000B587B0142102A8FDF721FF00BF5948C06A042108435749C8620846C06A04211D
:202380000840019000BF00BF00BF5248C06A802108435049C8620846C06A802108400190C2
:2023A00000BF00BF00BF4B48C06A012108434949C8620846C06AC007C00F019000BF00BFDD
:2023C00000BF0846C06A022108434249C8620846C06A02210840019000BF00BF01221C2151
:2023E00005200007FEF7FAFB00223B493B48FEF7F5FB012291023948FEF7F0FB00228121DE
:20240000090205200007FEF7E9FB02200290032003900020049002A905200007FEF7E4FAE4
:202420000C20029011200390002004900320059002A905200007FEF7D7FA1020029001202E
:202440000390002004900220059002A905200007FEF7CAFA012002901120039000200490C3
:20246000059002A91D48FEF7BFFA022002901C4803900120049002A91848FEF7B5FA194899
:2024800002900120039000200490059002A91348FEF7AAFA81200002029001200390002005
:2024A0000490059002A905200007FEF79DFA8020029000200390049002A90848FEF794FA99
:2024C000002201210520FEF7C7FC0520FEF7B8FC07B000BD001002400930000000040050BA
:2024E000000021100834000010B50E480E490860E1204002486000210B488160C1600161D2
:202500000C21416100218161C16101620020064948620846FFF776FB002801D0FDF73AFF70
:2025200010BD0000003801401409002010B5002425E013A000F070F900F002F900281DD11D
:20254000FF2101311348FDF783FF13480068134908400121490788420FD10F48406810497D
:202560000860084600680F4908600B49086880F3088800BF0B480068804710BDFDE7D8E705
:20258000C7EBB4ABCAE4C9FDBCB6CEC4BCFE0D0A0A000000384A0008005000080000FE2FC8
:2025A00018000020140000207047000010B5002819DA1A4A03071B0F083B9B089B00D258D5
:2025C0008307DC0EFF23A3409A438B071B0E8407E40EA3401A43114B0407240F083CA408A3
:2025E000A4001A5118E00E4A03231B02D21883089B00D2588307DC0EFF23A3409A438B0717
:202600001B0E8407E40EA3401A43054B032424021B198408A4001A5110BD00001CED00E0B2
:2026200000E100E0704770B505460C4606E0284600F0DCF8012801D1002070BD2046641E18
:202640000028F4D1401EF8E7F7B582B004460E460020306068460499FFF7E5FF002803D004
:202660000020C04305B0F0BD68460078182813D006DC012809D0022809D0042821D109E09E
:2026800041281BD061281CD119E080251CE00125AD0219E00020E5E768460499FFF7C3FF19
:2026A000002808D168460078182804D10020C04330600020D6E70020C043D3E700BF012091
:2026C000D0E70020C043CDE700BF68460078207001270AE0E0190499FFF7A5FF002802D0BB
:2026E0000020C043BEE7781C87B2681D8742F1DB6178A078FF225040814202D00020C043D1
:20270000B0E72946E01CFDF791FD0190E81C205C0002291D615C01430198814202D000208D
:20272000C0439FE7356000209CE7014608887047704710B50446204600F068F8002010BDE1
:202740003EB5002000900190029000243320FFF7F0FF174800F0DEFC0446002C17DD154867
:2027600000F05AF8144800F057F821466846FFF751FC12A000F050F8684600F04DF812A0A5
:2027800000F04AF813A000F047F800203EBD601C002801D10120F9E7A01C002801D10220BB
:2027A000F4E7E01C002801D10320EFE70420EDE730030020B8340008300700200A0D20532F
:2027C000697A653A200000002042797465730D0A000000002D2D2D2D2D2D2D2D2D2D2D2DFD
:2027E0002D2D2D2D2D2D2D0A0000000010B5044601231A4621460448FFF7C2FA002801D1A2
:20280000012010BD0020FCE71409002010B50446204600F041FC10BD10B5044603E0207891
:20282000FFF7F4FF641C20780028F8D110BD70B502460C460021002500231078302844D1BC
:202840005078782802D0507858283ED19078002800D170BD022131E0505C002802D123605B
:2028600001252DE0505C412802DB505C46280BDD505C612802DB505C662805DD505C3028FF
:2028800019DB505C392816DC505C302805DB505C392802DC505C30380AE0505C412805DB83
:2028A000505C462802DC505C373801E0505C57381E01831901E0002502E0491C0B29CBD30F
:2028C00000BF0B2936D3002534E000212CE0505C002802D12360012528E0505C6B2802D02D
:2028E000505C4B2805D1002903D09B02236001251CE0505C6D2802D0505C4D2805D1002972
:2029000003D01B052360012510E0505C302808DB505C392805DC0A205843565C303E8319D5
:2029200001E0002502E0491C0B29D0D300BF0B2900D3002528468CE700BF0278044B1B689C
:202940009A5C0270401C4A1ED2B2111EF5D170470800002010B5FEF74DF910BD00B599B028
:2029600034210CA8FDF723FC142107A8FDF71FFC1C216846FDF71BFC244800680321C9028F
:2029800088430121C902401820490860FEF76EFA1F4800690321C90288431D49086105207B
:2029A0000C90012000040D9000120E9002201590C1031691032189041791410518910CA8DB
:2029C000FEF70AFD002801D0FDF7E4FC0F20079003200890002009900A900B90012107A8EE
:2029E000FEF764FB002801D0FDF7D4FC81200090002002900320800406906846FEF740FAC9
:202A0000002801D0FDF7C6FC19B000BD007000404010024015480068FF2101310843134981
:202A200008600846C068124908401049C86008460068104908400D49086008468068400801
:202A40004000886008460068012189048843074908600846C068FD21090488430349C86086
:202A600000200861C803044988607047001002400C40FF88F6FFF6FE00ED00E0818CC9075E
:202A8000C90F002908D001684968012252049143826A1143026851600222416A1140022950
:202AA00007D101684968D2039143C26A1143026851600422416A1140042907D1016849689F
:202AC00012049143026B1143026851600822416A1140082907D10168496812039143426B51
:202AE0001143026851601022416A1140102907D10168896812029143826B1143026891604A
:202B00002022416A1140202907D10168896812029143C26B1143026891604022416A1140DA
:202B2000402915D10168496892039143026C11430268516001221205016C914208D101682A
:202B40004968032252059143426C1143026851608022416A1140802907D101684968120309
:202B60009143826C114302685160704738B504460020E067FEF738F8054620680068082146
:202B8000084008280BD114482B46002289040090204600F03FFA002801D0032038BD2068AD
:202BA00000680421084004280BD10B482B46002209050090204600F02DFA002801D003201B
:202BC000ECE720206067A06700BF00217020015500BF0020E2E70000FFFFFF0170B5054638
:202BE000AC6A00215A200153522001532046FEF722FF70BD01680968FF22213291430268D5
:202C000011600168896849084900026891602021816700210166704710B50446206800688D
:202C2000402188432168086020206067002060662046FFF7D5F910BDF0B587B0044610203D
:202C400004900025002003900026E7492068884200D100E000BF2169A068084361690843FE
:202C6000E1690843074620680068E049084038432168086020684068032109038843E16831
:202C8000084321684860A769D7492068884201D0206A0743206880680B21090288433843A4
:202CA0002168886000BFD249206888421CD1D148C0688007800F002806D001280AD0022808
:202CC00005D003280CD108E0012004900BE00220049008E00420049005E00820049002E0B6
:202CE0001020049000BF46E0C349206888421CD1C048C0680C210840002806D004280AD037
:202D0000082805D00C280CD108E0002004900BE00220049008E00420049005E0082004901F
:202D200002E01020049000BF25E0AF49206888421FD1B048C068032189020840002808D0D8
:202D400001218902401A0AD0401A05D0401A0CD108E0002004900BE00220049008E00420E3
:202D6000049005E00820049002E01020049000BF01E01020049000BF9B492068884256D1F8
:202D8000049804281AD004DC002807D002281CD108E0082816D0102817D117E0FEF790FAF7
:202DA000064616E0934840380068102108400009002801D0914E00E0914E0AE0FEF7A4FA80
:202DC000064606E00126F60303E000BF0120039000BF00BF002E0AD0606841004018B04272
:202DE00003D860680003B04202D201200390F4E0606802903046FF21013100F091FA626878
:202E0000520800238018594101910090029AFDF785F9054603200002854205D3794885423C
:202E200002D82068C560D8E001200390D5E00121C903E06988426FD1049804283CD006DCF3
:202E4000002809D0012813D002284AD11CE008283ED0102845D145E0FEF732FA4000616849
:202E60004908401802906168FDF742F985B23CE0FEF738FA40006168490840180290616898
:202E8000FDF736F985B230E05A4840380068102108400009002807D061684A085A4BD0181D
:202EA000FDF726F985B206E061684A08574BD018FDF71EF985B218E0FEF726FA40006168E5
:202EC0004908401802906168FDF712F985B20CE061684A0801231B04D018FDF709F985B259
:202EE00003E000BF0120039000BF00BF102D0FD3474885420CD846480F38284005902807A4
:202F0000400F05990843059005982168C86064E00120039061E0FFE7049804283AD006DCC3
:202F2000002809D0012812D0022847D11AE008283BD0102842D142E0FEF7C2F961684908D7
:202F4000401802906168FDF7D3F885B23AE0FEF7C9F961684908401802906168FDF7C8F876
:202F600085B22FE0234840380068102108400009002807D061684A08204BD018FDF7B8F82D
:202F800085B206E061684A081D4BD018FDF7B0F885B217E0FEF7B8F9616849084018029035
:202FA0006168FDF7A5F885B20CE061684A080123DB03D018FDF79CF885B203E000BF01200D
:202FC000039000BF00BF102D05D31148854202D82068C56001E00120039000202066606623
:202FE000039807B0F0BD000000480040F369FFEF00380140401002400044004000093D002B
:203000000024F400FFFF0F0000127A000048E801FFFF0000FFB581B004460D4617460A9E49
:2030200022E0701C00281FD0FDF7DEFD0499401AB04201D8002E17D120680068FF21A13162
:2030400088432168086020688068400840002168886020206067A06700BF00217020015577
:2030600000BF032005B0F0BD2068C0692840A84201D1012000E00020B842D2D00020F1E782
:2030800010B510200349096808620248FEF7D4FC10BD00001409002001B501231A46694612
:2030A0000348FEF71DFF00BF0248C06900BF08BD140900200038014010B503460C46194689
:2030C000E21DF93200BF49005200FF2001301040002800D0491C012000040840002801D009
:2030E000044841400120000410400028EBD088B210BD00002110000010B500BF03780C78F0
:2031000063400370401C491C531EDBB21A1EF5D110BD0000F0B5FFB0FFB099B00646002156
:203120000C910D910E910F91049100F02FF979490391002108910691059100BF0027002124
:203140000791109600BF7D22D20009A915A8FFF77BFA002802D0012871D1ADE0002106917D
:203160000998401C002802D001280ED107E00620FFF7DFFA00207FB07FB019B0F0BD06205A
:20318000FFF7D7FA0120079094E010A8407DF9B2884203D01520FFF7CCFA8AE0002F4FD1D5
:2031A00010A8C07D002843D0002515AC033405E0207829466D1C584A5054641C20780028C7
:2031C00001D0FF2DF4DD002029466D1C524A50540025641C05E0207829466D1C11AA505450
:2031E000641C2078202801D00F2DF4DB002029466D1C11AA505404A911A8FFF718FB47491D
:203200000498884208D91820FFF793FA1820FFF790FA0020C043AEE74049891E3D48FDF793
:2032200017F90620FFF785FA4320FFF782FA3DE00620FFF77EFA0121079108913AE044E0CC
:2032400015A90331099A1098FCF798FF0B9600210A910AE00CA90B9800F0CEF80B98014668
:2032600010310B910A9810300A9009990A988842F0DB0296099881B2C8170191810F019816
:203280000818821003A8049B0299FDF785F8002803D10620FFF74DFA08E01820FFF749FA6E
:2032A0001820FFF746FA0120C04364E77F1C0121059100BF00BF1DE01820FFF73AFA1820C9
:2032C000FFF737FA0220C04355E70598002802DD0698401C06900698052807DD1820FFF755
:2032E00028FA1820FFF725FA002044E74320FFF720FA00BF00BF0798002800D123E700BFC2
:2033000000BF0898002800D118E700BF00BF049831E70000005000083007002001AC0000C8
:20332000F8B582B28BB2040C0D0C10465843002126465E43370C36048019794116466E434A
:20334000370C36048019794126466E438919F8BD30B47446641E2578641CAB4204D3635D68
:203360005B00E31830BC18471D46F8E702E008C8121F08C1002AFAD170477047002001E05A
:2033800001C1121F002AFBD17047000000B5124812490860124813490860084601680F488F
:2033A0000068FCF772FF10481049086008460068FCF786FF08480E49086008460068FEF740
:2033C0004FFF07480B4908600846016807480068FCF7A0FF00BD0000300000200000002067
:2033E00030010020040000203002002008000020100000200C00002030B504460D46FFF70A
:20340000C5FF102221460948FCF799FF084801682046FEF737FE102229462046FFF76CFEC3
:20342000102202492846FCF78AFF30BD30020020100000200024FDF7E5FBFFF78FFAFEF74A
:203440008FFFFEF77BFFFFF74FF80CE00648FFF76CF904460548844202D1FFF767F802E036
:203460000348FEF7C1FDF1E7384A0008AAAA000000500008210504198912130018DECA018E
:20348000305201231305331993070800205BA34A21BAF9FC0000000000000000010203043E
:2034A000060708090000000001020304030406080C101820300000000A0A0D2050726F6772
:2034C00072616D6D696E6720436F6D706C65746564205375636365737366756C6C79210AF4
:2034E0000D2D2D2D2D2D2D2D2D2D2D2D2D2D2D2D2D2D2D2D2D2D2D2D2D2D2D2D2D2D2D2D4C
:203500002D0D0A204E616D653A2000002C35000800000020300000006C3300085C35000873
:2035200030000020101000007C330008000000000000000000000000000000000000000064
:1C354000000000000000000000000000000000000000000000000000000020004F
:20500000381F0020D5500008BD9200087F8900080000000000000000000000000000000085
:205020000000000000000000000000000D970008000000000000000039930008B997000898
:20504000E7500008E7500008E7500008E7500008E75000085D5C0008E7500008E7500008D6
:2050600000000000E7500008655B0008E7500008E7500008D58D000800000000E750000802
:2050800000000000E75000080000000000000000E750000800000000E7500008E750000814
:2050A000E7500008E7500008E750000891A60008E7500008E7500008000000000000000076
:2050C0000348854600F098FC0048004785B60008381F00200448804704480047FEE7FEE77D
:2050E000FEE7FEE7FEE7FEE779980008C150000830B50B46014600202022012409E00D46AA
:20510000D5409D4205D31D469540491B2546954040191546521E002DF1DC30BD70B5002493
:205120002546002801DA01244042002901DA01254942FFF7DDFFAC4200D04042002C00D097
:20514000494270BDF0B51FB40646002082B005464024019100901BE0019922460F463046E8
:2051600000F086FB049A059B801A994110D310461946224600F06CFB361A8F410197224695
:2051800001200021009F00F063FB38184D4100902046641E0028DFDC019B0098294632468C
:2051A00007B0F0BD03460B439B0703D009E008C9121F08C0042AFAD203E00B780370401C9D
:2051C000491C521EF9D27047D2B201E00270401C491EFBD270470022F6E710B513460A46ED
:2051E00004461946FFF7F0FF204610BD30B504460020034600E05B1C934203D2E05CCD5CF0
:20520000401BF8D030BDF8B502464A40D40F42004B0052085B089A4202D202460846114635
:205220004A0023D0C30D4A00DDB2120EAD1A202D35DA49020126490AF6058A19002C00D0E6
:20524000524220214F1B1146B9402A411018C20D9A4221D0002C17D0012D08DCDA05801AF2
:20526000D20F8019D207DBB200F02EFBF8BDDA05801A012340001B06C01880185A428018DE
:20528000CA0F1043490007E04908C2071143DA05801A80194008801800F00EFBF8BD610043
:2052A0000122511A001BF7E70122D2075140AAE70122D2075040A6E7024670B54A40D30F57
:2052C000DB0740002DD04A002AD0010E140E000212020919400A520A8418E50104465443F9
:2052E000000A120A2E045043A4194219200CC543AA18120C0125AD03521C521912047F391A
:20530000240400D0521C104301D44000491EC2B20C06C0092018401C4008802A02D003E0CE
:20532000002070BD40084000002900DA0020184370BD70B502464A40D50F40004A00ED0794
:2053400040085208002814D0002A12D0C40DD30D41020120C0055202490A520AE41A091897
:2053600012187D34914201D3641C00E04900002C01DA002070BD0023914201D3891A0343FB
:20538000400849000028F7D100290AD0914202D10121C90705E0914201D2012101E0012141
:2053A000C943E005C018401900F086FA70BD0000F0B507460846584087B0C00F0490480074
:2053C0000E46590040084908BC1A884105D2384631461E4617460B460246580040081043CF
:2053E0004CD0300D039040055900400D490D0590401A0290402872DA18030121000B0905F5
:205400000843019004980092002805D0019952420020884100920190029840210A1A019992
:20542000009800F015FA05460C466B4607CB00F030FAC0197141039A0E0D0023D7175640B1
:205440001A467A40164344D0049A002A2DD0029A012A039A15DC1205C01A91410126360586
:20546000001C7141D20F059ED2070093019202962A46234600F06EFA07B0F0BD38463146B9
:20548000FAE71605224A0F46B218C01AB74101210905001C4F4100187F41114618187941BE
:2054A000E20F10436D19644113E0E2076D0815436408C2071443039A01261205C01A9141C1
:2054C0003605001C7141CE07400830434908C01851412A46234600F030FACDE7FFE704984F
:2054E00001224000C117121A00238B4104983146C417381AA141EEE730B40124E4076340C8
:2055000030BC55E730B40124E407614030BC4FE70000E0FFF0B51FB488B00B9909980024B4
:2055200048400999C00F490049080991C0070B990090490049080B9109990898A646084394
:205540001CD00B990A98084318D0099801244000420D4800410D099824050003000B2043C0
:2055600009900B980003000B20430B9050181C494018002201901446104605E0002001460F
:205580000DB0F0BD032801DA034600E003239C46C11A0AAE0AE05F0008ADED5B4F00F75BF0
:2055A0007D430027AA187C41491C5B1E6145F2DD410004AB5A522104120C0A43240C401C7A
:2055C0000828DFDB019802900099704601910090059B049A0799069800F0BCF9D0E700006D
:2055E0000DFCFFFFF0B50C465C4085B0E40FE40703944C00002664085900944649080246BD
:205600000296224321D062460A431ED06200570D4A000E032303550D012402462C49240505
:20562000781B1B0B360B401823432643614600901C46501AB44103D30098401C009002E015
:20564000921800985B41002803DA0020014605B0F0BD0020012109050746864611E064469A
:205660001D46141BB54106D36546521BB341744607430C43A646CD074008490828439218FC
:205680005B4105460D43EAD11046184313D06046194650407140084306D06046101AB34159
:2056A00006D20122002306E000220123DB0702E00122D2435310009874460105381C6141F3
:2056C000029C039D0019694100F037F9BFE70000FD030000C217C10F504010B54018CA07DC
:2056E0009623002100F0F0F810BD10B500229623114600F0E9F810BD0EB5C217C10F50409A
:20570000CA0740180021054B0293019200910A460B4600F01FF903B000BD000033040000E6
:205720000EB505490291002100910A460B46019100F010F903B000BD3304000041004002BD
:205740000122400AD205090E80187F2901DA00207047962903DC9622511AC84070479639AD
:20576000884070474A0009030123090B1B051943094B10B5520D9A4201DA002010BD064B33
:2057800034339A4203DC9A1A00F072F810BD03495118884010BD0000FF030000CDFBFFFFFA
:2057A000C20FD207400040080BD0C10D0723DB01C91840020905400A1143C20840071143D4
:2057C000704700200146704710B5002904DB0124E40740428C412146002B04DB1C460123D1
:2057E000DB075242A341994200D1904210BD0000CB0FDB07490010B5490802460A4307D07D
:205800000A0D07240903E401090B121B002A01DC002010BDC900440F0C43C100E018D20525
:20582000801800F049F810BD0122D207002800DB101A002900DB511A814270470122D207C4
:20584000002800DB101A002900DB511A8842704710B5202A04DB0146203A9140002010BDDE
:20586000914020239C1A0346E3401943904010BD10B5202A04DB0846203AD040002110BD65
:205880000B46D340D0402024A21A91400843194610BD10B5202A06DBCB170846203A104181
:2058A000C1170B4306E00B461341D0402024A21A91400843194610BD002904DA401C490033
:2058C00001D140084000704770B40024050C05D11024000402D1002921D01124050E01D149
:2058E00000020834050F01D10001241D850F01D18000A41C002801DB4000641C002908D0D7
:2059000020252E1B0D46F540A14000D001212943084301061B1B000ADB1D02D5002070BC85
:205920007047DB05181880180029F8DA401C4900F5D170BC40084000704710B5002B08DA65
:205940000024401C614192185B411A4301D14008400010BDF0B51FB482B005460C0003D087
:20596000084604F0A5FF02E004F0A2FF20300246009021462846FFF76BFF049B059A0446E5
:205980000F4618431143084314D0184610431BD0009840210A1A18460599FFF769FF054676
:2059A0000E46009A05990498FFF752FF084305D0012004E02046394607B0F0BD0020C11712
:2059C00005430E432C43374300990E986305401A7905E40A00220C43FD0A0A3002D500202F
:2059E0000146E9E70105101969410C9C0D9D00196941FFF7A2FFDFE7064C0125064E05E094
:205A0000E36807CC2B430C3C98471034B442F7D3FFF75AFBE0B9000800BA000870B58C1858
:205A20000578401C6B075B0F01D10378401C2A1106D10278401C03E006780E70401C491C80
:205A40005B1EF9D12B0705D40023521E0DD40B70491CFAE70378401CCB1A921C03E01D78E1
:205A60000D70491C5B1C521EF9D5A142D8D3002070BD000038B50446074908480068FFF77F
:205A800037FB6043009002E00098401E009000980028F9D138BD000040420F0050010020B8
:205AA00070B504460025206880688007800F012807D120680068C007C00F002801D001202B
:205AC00000E00020002839D1206880681C490840002801D1012000E00020002809D1606D8D
:205AE000102108436065A06D01210843A065012070BD206880680121084321688860012029
:205B0000FFF7B8FF01F0ECF805460EE001F0E8F8401B0A2809D9606D102108436065A06D6F
:205B200001210843A0650120E2E720680068C007C00F0121484048400028E7D00020D7E794
:205B40001700008010B502460B460020002103E0545C2418A0B2491C9942F9D3C443A0B289
:205B600010BD000010B5034800F0B8FD024800F0B5FD10BDD81A0020901A002030B51C25E8
:205B8000446C2C400125A540046C6560046863608468102C04D10468A2600468E16003E07F
:205BA0000468A1600468E26030BD000010B501201749487202201749487203201649487265
:205BC000042016494872124815490978017012481349097801700F4811490978017004226D
:205BE00010490B48401DFFF7DDFA04220D490A48401DFFF7D7FA04220A490648401CFFF7C4
:205C0000D1FA042207490548401CFFF7CBFA10BD84150020BE150020A615002098150020BE
:205C2000270100201C01002010B503F071FC202003F0B0FD012005F02FFA002003F0AAFDE1
:205C4000044805F0BFF8044805F0A4FB002005F0E1FB10BD600000208380000010B5012144
:205C60000520000701F02CF8002802D000200A4908600221094801F023F8002805D1084840
:205C800000880A21484307490880012000F012FF022000F00FFF10BD480100200004005022
:205CA00036010020400100207047000000210A4A51610A494968012252021143074A51607D
:205CC0001146496808221143044A51600021C209D201116070470000201B0020002002409B
:205CE0007FB504460D460020039000F09BFE002000900194E809029003A9684600F014FE73
:205D0000002804D000F056FE002004B070BD00F051FE0120F9E710B50346002002E01C5C7A
:205D20000C54401C9042FAD310BD0000002039498969FF2201321140914208D13649496925
:205D400002221143344A5161FF210131084331498969012252021140914208D12E494969F5
:205D6000012211432C4A516101214902084329498969012292021140914208D12649496993
:205D800008221143244A5161012189020843214989690122D2021140914208D11E49496904
:205DA000042211431C4A51610121C902084319498969012252031140914208D1164949693F
:205DC00010221143144A516101214903084311498969012252041140914207D10E494969AA
:205DE000202211430C4A51612021084309498969012212041140914208D10749496940229B
:205E00001143054A5161012109040843014988617047000000200240201B002070B504469D
:205E200000F05EFF05460BE0601C002808D0002C04D000F055FF401BA04201D9032070BDB8
:205E40001F488069C007C00F0028EDD11C48806902210840022801D119498861184880692E
:205E6000FF2101310840884223D0154880694900084088421DD0124880694900084088429F
:205E800017D00F48806949000840884211D00C4880698900084088420BD0094880690901A8
:205EA0000840884205D00648806949100840884203D1FFF73BFF0120C1E70020BFE70000C6
:205EC00000200240F0B585B006460F4614460025029601970020009000F0A4FD13E0019869
:205EE000006803900220039A029900F073FD00900098002800D008E00298001D0290019803
:205F0000001D01902D1DA542E9D300BF00F052FDA54202D2002005B0F0BD0120FBE70000A8
:205F200010B50B4800F070FB0A21094800F0F6FA074800F09DF9012149020840884204D169
:205F4000034800F098F980B210BD00BFFCE700002C190020F0B587B000220121404800F0D7
:205F6000B8FEFFF7DDFF0546FFF7BFFB04463D49FFF7DFF93C49086001221146384800F029
:205F8000A8FE39480068FFF70BFC04460022374BFFF71AFC5DD836480078002821D0002017
:205FA00033490870FFF7BCFF0546FFF79EFB04462C49FFF7BEF92C49086008460068FFF76D
:205FC000EFFB04460022294BFFF796FA0022294B05910490FFF79EFA0646FFF709FC26496D
:205FE000086021480068FFF7DBFB064600221F4BFFF782FA0446214A214BFFF78BFA039122
:2060000002901D480068FFF7CBFB04461B4A52421C4BFFF77FFA01910090039B029AFFF7FA
:20602000C7F905910490FFF7E3FB13490860164911480068FFF702FC02D213480E490860DC
:2060400000210D480068FFF7EFFB02D200200A49086009480068FFF771FBC0B207B0F0BDE2
:206060000004005000401B442800002000000C403000002000E064402C00002033333333AD
:2060800033B33040CCCCEC3F0000C842F8B5044600250026002700BF5020005D012801D1ED
:2060A0000220F8BD01215020015500BF206880688007800F012806D120680068084000287C
:2060C00001D0012000E00020002841D1606DFF21013188430221084360652068C068870739
:2060E000BF0F2068C068800880002168C860206880680121C90708432168886000F0F0FD6E
:20610000064611E000F0ECFD801B0A280CD9606D0221884310210843606500BF002150206B
:20612000015500BF0120BCE720688068C00FC0070121C9078842E5D02068C068384321685B
:20614000C860606D0221884301210843606504E0606D202108436065012500BF00215020B2
:20616000015500BF28469CE770B504460D4600BF5020005D012801D1022070BD01215020EF
:20618000015500BF2068806804210840800800280AD0606D20210843606500BF0021502015
:2061A000015500BF0120E8E72D496868884229D02068806A29684903490B08432168886270
:2061C00028684003400B2749084001218904884208D12548806849010843234988600A202F
:2061E000FFF748FC28684003400B204908400121490488422CD11C488068490108431A491C
:20620000886025E02068806A29684903490B88432168886228684003400B124908400121CD
:206220008904884205D110488068490188430E49886028684003400B0C4908400121490473
:20624000884205D108488068490188430649886000BF00215020015500BF00208DE7000021
:20626000011000000000044800270140000002440146486D704701460868006C7047000086
:2062800010B50446002C01D1012010BD606D002806D1A065002150200155204600F00EF9EE
:2062A000606D10210840102806D02068806804210840800800280AD0606D10210843606515
:2062C00000BF00215020015500BF0120DDE7606DFF210131884302210843606520688068E7
:2062E0008007800F012807D120680068C007C00F002801D0012000E0002000283AD100BFF5
:20630000032189076068884207D049426068884203D04900606888420CD120680069800047
:2063200080082168086120680069616808432168086112E02068006980008008216808610F
:206340005C4880680F21890488435A49886008468068616808435749886000BF2068C0685D
:20636000182188432168C8602068C068A16808432168C8604F4880680121490688434D4962
:20638000886008468068A18E490608434949886020688068012109070840002804D120682D
:2063A00080680843216888602068C068424908402168C8602169E068022901D1042100E031
:2063C000002108432021095D490308432C21095D49000843216B0843A16989030843E169CA
:2063E000C90308432168C96808432168C860FF21C231606A884207D0A16A606A08432168A9
:20640000C96808432168C8602120005D012813D12020005D002807D12068C0680121090428
:2064200008432168C86007E0606D202108436065A06D01210843A065E06B012817D12068F8
:206440000069FF218900884321680861216C606C0843A16C08432168096908432168086139
:206460002068006901210843216808610BE020680069C007C00F002805D020680069400824
:2064800040002168086120684069C008C0002168486120684069A16B084321684861002005
:2064A000A065606D022188430121084360650020EBE60000002701401902FEFF10B586B07E
:2064C0000446142101A8FEF786FE1249206888421ED11148406B491508430F49486300BF10
:2064E0000846C06A012108430B49C8620846C06AC007C00F009000BF00BF02200190032047
:2065000002900020039001A90520000700F0E2FA06B010BD0024014000100240F8B5044663
:206520000D46002600276069082801D1082711E02068C068C007C00F00280AD0606D20217A
:206540000843606500BF00215020015500BF0120F8BD0C2700F0C4FB064614E0681C002822
:2065600011D0002D04D000F0BBFB801BA8420AD9606D04210843606500BF00215020015583
:2065800000BF0320E4E72068006838400028E5D0606D01214902084360652068C0680321EB
:2065A00089020840002826D12020005D002822D1206800680821084008281CD12068806843
:2065C00004210840800800280DD1206840680C21884321684860606DFF210131884301215B
:2065E0000843606507E0606D202108436065A06D01210843A065A069002802D10C2021684E
:2066000008600020A4E7000070B5044600252068806804210840800800282BD100BF50201B
:20662000005D012801D1022070BD01215020015500BFE069012803D02046FFF731FA0546F5
:20664000002D18D1606D0D490840FF210131084360650020A06500BF00215020015500BFCD
:206660001C202168086020688068042108432168886000E002252846D6E70000FEF1FFFF7D
:2066800070B5044600252520005D022803D00420E063012520E0206800680E2188432168C7
:2066A00008602068006840084000216808601C21606C084001218140206C41600121252041
:2066C000015500BF00212420015500BFA06B002802D02046A16B8847284670BD70B50446DB
:2066E000206C0568206806681C20616C014004208840284000281DD004203040002819D053
:206700002068006820210840002805D12068006804218843216808601C21606C08400421BB
:206720008140206C4160206B00285AD02046216B884756E01C20616C0140022088402840FB
:20674000002825D002203040002821D02068006820210840002808D1206800680A21884311
:20676000216808600121252001551C21606C084002218140206C416000BF0021242001558F
:2067800000BFE06A00282CD02046E16A884728E01C20616C0140082088402840002820D08A
:2067A0000820304000281CD0206800680E218843216808601C21606C084001218140206C92
:2067C00041600120E06301212520015500BF00212420015500BF606B002802D02046616BC7
:2067E000884770BD70B50446002C01D1012070BD244A2168881A1421FEF77AFC8000606465
:20680000204808382064022125200155206805681D480540E168A0680843216908436169B4
:206820000843A1690843E1690843216A084305432068056001218903A068884217D0114858
:206840007830806A1C22616C11400F228A4090430C49783188621C22616C114060688840A8
:2068600008497831896A08430649783188620020E063012125200155002124200155002003
:20688000B5E70000080002400F80FFFFF8B504460D4616461F460020009000BF2420005D6A
:2068A000012801D10220F8BD01212420015500BF2520005D01282DD10221252001550020E4
:2068C000E0632068006840084000216808603B46324629462046FFF751F9206B002806D075
:2068E000206800680E210843216808600BE0206800680421884321680860206800680A2166
:2069000008432168086020680068012108432168086006E000BF00212420015500BF0220AC
:2069200000900098BFE70000F8B504460E460127002500BF1C48007C012801D10220F8BD80
:2069400001201949087400BF1848FFF767FA0746002F22D1401E3060656817E02846FFF73D
:20696000A5F91248FFF75AFA074611484068082188430F49486008464068491588430C491F
:206980004860002F01D0356006E08035A068C00161684018A842E1D800BF00BF00200249A9
:2069A000087400BF3846CAE7201B002050C300000020024006484068022108430449486044
:2069C0000846406801210843014948600020704700200240F8B507460C461546012600BF9C
:2069E0000E48007C012801D10220F8BD01200B49087400BF0A48FFF711FA0646002E06D19F
:206A00000649486125600648FFF708FA064600BF00200249087400BF3046E6E7201B002064
:206A200050C300001D484068C007C00F002816D000BFEFF31080014600BF72B61848174A72
:206A4000D0601848D06000BF81F3108800BF10464068C007C00F002801D0012070470F4830
:206A6000406802221040022815D100BFEFF31080014672B60C48094A10610C48106108461F
:206A800080F3108800BF1046406802221040022801D10120E2E70020E0E70000002002408B
:206AA000EFCDAB8905040302BFAE9D8C161514137047000010B504460548406920400028AC
:206AC00004D0034844612046FFF7F2FF10BD00000004014070B50346002200240020DAE005
:206AE000012696400D6835402C46002C77D04D68022D02D04D68122D15D1D508AE001D464C
:206B00002035A8595507EE0E0F25B5400646AE4330465607F60E0D69B5402843D508AD002A
:206B20001E46203670514D68012D08D04D68022D05D04D68112D02D04D68122D18D19868C4
:206B400056000325B5400646AE4330465600CD68B540284398605868012595400646AE4334
:206B6000304610264D6835402D09954028435860186856000325B5400646AE4330460D79E5
:206B8000AD07AD0F5600B54028431860D86856000325B5400646AE43304656008D68B540B1
:206BA0002843D860012636074D683540B54271D13C4D6D6B012635433A4E75633A4D9608E6
:206BC000B600A85995072E0F0F25B5400646AE43304605252D07AB4202D1002515E059E0D8
:206BE000324DAB4201D101250FE0314DAB4201D102250AE02F4DAB4201D1032505E02E4D31
:206C0000AB4201D1052500E006259607360FB5402843254D9608B600A851284D286805462F
:206C2000A5432846012636044D683540B54202D1054625432846214D286068680546A5438F
:206C40002846012676044D683540B54202D1054625432846194D6860A8680546A543284631
:206C6000012636054D683540B54202D1054625432846124DA860E8680546A543284601261E
:206C800076054D683540B54202D10546254328460A4DE860521C0D68D540002D00D01FE7CA
:206CA00070BD000000100240080001400004005000080050000C0050001C00500004014053
:206CC000024613690B40002B01D0012000E000207047002A01D0816100E08162704700007A
:206CE00001480068704700004C01002002480068401C0149086070474C01002010B50024F2
:206D0000084800684021084306490860002000F00BF8002801D0012401E000F0E1F9204616
:206D200010BD00000020024070B5044600257D21C90009480068FEF7DBF9064601F066FB09
:206D4000002801D0012504E000222146501E00F0EFF9284670BD00005001002070477047E7
:206D600070B505461F480078401C1E49087001201D4908701D4800881D49098840181B49EA
:206D80000880084600881B49884203DD1A48008816490880154800881849096848611849F5
:206DA000C888FEF7A2FC06461649FEF7C2FA0446154801682046FEF726FA134908601049EC
:206DC000488FFEF792FC04460F4801682046FEF72BFD05D20D480078002801D004F0CEFC71
:206DE00070BD000046010020E6000020300100203201002029810000340100208819002095
:206E0000840D002000007A444801002038010020704710B50446002C01D1012010BD02216C
:206E20002E200155204601F0DDFF204600F0F4F800212E20015500BF2D20015500BF002033
:206E4000ECE77047704710B5044620680068C007C00F01214840484000280CD020688068B6
:206E6000084048404840002805D00120216848602046FFF775FF20680068022108404008F8
:206E800000280BD02068806808404008002805D00220216848602046FFF760FF20680068F4
:206EA00004210840800800280BD02068806808408008002805D0042021684860204600F0F2
:206EC0000DF92068006808210840C00800280BD0206880680840C008002805D00820216852
:206EE00048602046FFF794FF2068006810210840000900280BD0206880680840000900289D
:206F000005D01020216848602046FFF728FF2068006820210840400900280BD02068806883
:206F200008404009002805D02020216848602046FFF788FF20680068402108408009002825
:206F40000BD02068806808408009002805D04020216848602046FFF774FF10BD70B504467C
:206F6000002C01D1012070BD6068012800D100BF26496069884200D000BF2E20005D0028E0
:206F800005D100212D200155204600F059F802212E2001552068C5686068012803D08905E2
:206FA000A06A884203D11E2128468843054617496069884201D01648054016480540A16853
:206FC00060680843216A0843616A0843A16A084305436068012804D00121C905A06A88428B
:206FE00003D1E16820690843054308496069884205D06169A0690843E1690843054320681C
:20700000C56001212E2001550020ACE7FFFF00003F1FFFFFF8F119FF10B504460649206891
:20702000884208D10548806B40004008034988630D2000F065F810BD007C00400010024061
:2070400010B504460949206888420DD10848806B4905084306498863002201210D2000F030
:2070600067F80D2000F058F810BD0000007C00400010024001460868C069704710B50346C4
:2070800002242E20C4541448006824072043124C20601868C0680124E40420431C68E06058
:2070A00018688068012420431C68A06018680069012420431C682061186881611868426161
:2070C00018680069042420431C68206101242E20C454002010BD00000004014070470000C3
:2070E0000648406B01210843044948630846806B0904084301498863704700000010024063
:2071000000BFC206D20E01219140024A116000BF7047000080E100E000BFC206D20E012118
:207120009140024A116000BF7047000000E100E070B504460D4616462946204602F0C0F8ED
:2071400070BD0000024949688143014A516070470070004003480068FF2101310843014945
:207160000860704700700040024949680143014A5160704700700040074800680221084378
:207180000549086005480069042108430349086100BF00BF30BF70470070004000ED00E0BD
:2071A00010B5024600200E4B1868800880000346134318460A4B18600A4B1B690424234390
:2071C000084C2361012901D130BF02E040BF20BF20BF044B1B690424A343024C236110BDCD
:2071E0000070004000ED00E0F8B5044620212068084020287CD120680840202800D100BFCD
:2072000000278148806B012109070840002805D17D48806B08437C49886301277B4800681D
:20722000FF2101310840002816D178480068084376490860FFF754FD064606E0FFF750FD4F
:20724000801B642801D90320F8BD70480068FF21013108400028F1D06B4805680321090560
:207260000D4060680840A8420DD0091160680840884208D164480068012149040840884288
:2072800001D10120E0E76048403000690321090408400546002D3DD060680840A84239D0B2
:2072A000202120680840202834D1574840300069032109048843054653484030006901211B
:2072C000C9040843504940310861084600690121C90488434C4940310861084605618015FA
:2072E00028408915884215D1FFF7FAFC064608E039E0FFF7F5FC801B4549884201D90320C8
:20730000A2E7414840300069012149020840400A0028EED000BF00BF0321090460680840DE
:2073200088420AD13848006809018843032212056168114008433449086000BF32484030BC
:207340000069032212046168114008432E494031086100BF012F05D12B48806B8905884357
:207360002949886300BF2078C007C00F002809D025484030C06880088000A16808432249F6
:207380004031C860022120680840022809D11E484030C0680C218843E16808431A494031FF
:2073A000C86004212068084004280AD116484030C068032189028843216908431249403198
:2073C000C86008212068084008280AD10E484030C068032109038843616908430A494031BF
:2073E000C86080212068084080280AD106484030C068032189048843A169084302494031FE
:20740000C860002020E70000001002400070004088130000F8B504460D46002C01D1012017
:20742000F8BD79480068C007C00FA8420ED27648006840084000284373490860084600681B
:20744000C007C00FA84201D00120E9E7022120680840022807D16D48C068F0218843A16833
:2074600008436A49C8602078C007C00F00284CD06068022809D165480068012149040840DC
:20748000400C002824D10120CAE76068032809D15E480068012149060840400E002817D1BF
:2074A0000120BDE76068012808D15848006804210840800800280BD10120B1E75348006880
:2074C000012149020840400A002801D10120A7E74E48C06880088000616808434B49C8606E
:2074E000FFF7FEFB0646606802280FD107E0FFF7F7FB801B4649884201D9032090E74348BD
:20750000C0680C2108400828F1D134E0606803280FD107E0FFF7E4FB801B3D49884201D974
:2075200003207DE73948C0680C2108400C28F1D121E0606801280FD107E0FFF7D1FB801B9A
:207540003349884201D903206AE73048C0680C2108400428F1D10EE007E0FFF7C1FB801B72
:207560002B49884201D903205AE72848C0680C2108400028F1D124480068C007C00FA84244
:207580000ED9214800684008400028431E49086008460068C007C00FA84201D001203FE723
:2075A000042120680840042808D11848C068072109028843E16808431449C8600821206881
:2075C0000840082809D11148C0680721C90288432169C90008430D49C86000F049F80B4979
:2075E000C968F022114009090A4A515CC8400A4908600020FFF798FB0746002F01D03846AD
:207600000EE700200CE70000002002400010024088130000BEB90008500100200148006872
:20762000704700005001002000B5FFF7F7FF0549C968072212021140090A034A515CC8405F
:2076400000BD000000100240CEB9000800B5FFF7E5FF0549C9680722D2021140C90A034A10
:20766000515CC84000BD000000100240CEB90008FEB52E48C7680C203840002845D0042852
:2076800004D008280CD00C283ED10BE02748006810210840002801D0254C00E0254C41E0B0
:2076A000254C3FE00F2080043840800C23490E5C032080053840800D401C01901B48C06888
:2076C000012109040840002807D01B49714308460199FDF70DFD054614E014480068102102
:2076E0000840002807D01249714308460199FDF7FFFC054606E00F49714308460199FDF744
:20770000F7FC05462C460DE000BF08484068072149030840400B00900098401C01218140A7
:20772000CC0300BF00BF2046FEBD00000010024000093D000024F40000127A00D6B9000808
:20774000FEB50446002C01D10120FEBDF848C6680C210E40C768012109040F402078C0075D
:20776000C00F002872D0082E04D00C2E0FD1084687420CD1EE480068012149040840400C17
:20778000002863D06068002860D10120DDE700BF012109046068884205D1E5480068084352
:2077A000E349086027E005210904606888420ED1DF480068012189040843DD490860084625
:2077C0000068012109040843D949086013E0D8480068012109048843D5490860084600688C
:2077E000012109040840009000BFD148006889008843CF49086000BF6068002813D0FFF7E6
:207800006FFA054606E0FFF76BFA401B642801D903209AE7C6480068012149040840400C95
:207820000028F0D012E0FFF75BFA054606E0FFF757FA401B642801D9032086E7BC480068EE
:20784000012149040840400C0028F0D102212068084002287AD1E0680290042E03D00C2EBB
:2078600034D1002F32D1B2480068042108408008002804D00298002801D1012065E7AC4889
:2078800040681F2109028843216909020843A8494860084600680921884302990843A44933
:2078A0000860FFF7E5FEA249C968F02211400909A04A515CC840A04908600020FFF734FAC2
:2078C00001900198002841D001983EE70298002824D09748006809218843029908439449D2
:2078E0000860FFF7FDF9054606E0FFF7F9F9401B022801D9032028E78D48006804210840E0
:2079000080080028F1D08A4840681F21090288432169090208438649486017E084480068E4
:207920004008400082490860FFF7DAF9054606E0FFF7D6F9401B022801D9032005E77C489B
:2079400000680421084080080028F1D1102120680840102867D1002E36D1754800684901CB
:207960000840400A002804D0A069002801D10120EBE66F484068072149038843216A084310
:207980006B494860084640680002000A217F0906084367494860206A400B401C0121814023
:2079A000C8036349C968F02211400909614A515CC840614908600020FFF7B6F90190019849
:2079C00000284BD00198C0E6A06900282CD058480068FF210131084355490860FFF780F9DE
:2079E000054606E0FFF77CF9401B022801D90320ABE64F480068012149020840400A0028B2
:207A0000F0D04B484068072149038843216A084347494860084640680002000A217F09066D
:207A200008434349486019E041480068FF21013188433F490860FFF753F9054606E0FFF767
:207A40004FF9401B022801D903207EE638480068012149020840400A0028F0D10821206877
:207A60000840082839D1606900281BD0304840300069012108432E4940310861FFF730F97A
:207A8000054606E0FFF72CF9401B022801D903205BE62748403000690221084040080028B4
:207AA000F0D01AE022484030006940084000204940310861FFF714F9054606E0FFF710F9CB
:207AC000401B022801D903203FE61948403000690221084040080028F0D104212068084034
:207AE000042879D1002000901148806B89060840002806D10E48806B08430D498863012058
:207B000000900E480068FF210131084000281ED10A480068084309490860FFF7E1F805468D
:207B20000EE0FFF7DDF8401B642809D903200CE600100240BEB900085001002000700040BC
:207B400085480068FF21013108400028E9D000BFFF210131A068884205D180480069084340
:207B60007E49086130E0A06800280DD17B480069FF2101318843794908610846006909156E
:207B80008843764908611FE005210902A06888420DD1724800690121890208436F490861D6
:207BA00008460069891508436C4908610CE06B480069FF2101318843684908610846006911
:207BC000091588436549086100BFA068002815D0FFF786F8054608E031E0FFF781F8401B4F
:207BE0005F49884201D90320AFE55C480069012149020840400A0028EFD013E0FFF770F83E
:207C0000054607E0FFF76CF8401B5549884201D903209AE551480069012149020840400A98
:207C20000028EFD10098012808D14C484038806B01210907884349494039886300BF606A4F
:207C400000284CD00C2E69D0606A022848D14348403800680121090688434049403908608F
:207C6000FFF73EF8054606E0FFF73AF8401B022801D9032069E539484038006801214906DD
:207C80000840400E0028EFD1E16AA06A0843216B084332494039C968FD2212049143084376
:207CA0002E494039C860084600680121090608432A4940390860FFF713F8054606E0FFF7FE
:207CC0000FF8401B022801D903203EE5234840380068012149060840400E0028EFD038E0A7
:207CE0001E48403800680121090688431B4940390860FEF7F5FF054606E0FEF7F1FF401BA3
:207D0000022801D9032020E5144840380068012149060840400E0028EFD11AE0606A01281F
:207D200000D112E50D484038C768012000043840A16A88420BD10F2080043840E16A8842F1
:207D400005D1032080053840216B884201D00120FBE40020F9E400000070004040100240C7
:207D60008813000010B50446002C01D1012010BD606A002800D100BF0021A1625120005DF9
:207D8000002804D150200155204600F035F8022151200155206800684021884321680860A6
:207DA000A16860680843E1680843216908436169084301225202A16911400843E169084377
:207DC000216A0843A16A084321680860A069000C04210840616A0843216848602068C0690C
:207DE000910088432168C861002060650121512001550020BBE7000010B586B0044614216B
:207E000001A8FDF7E8F914492068884222D11348406B891408431149486300BF0846C06A18
:207E2000012108430D49C8620846C06AC007C00F009000BF00BFE0200190022002900020D4
:207E40000390032004900020059001A905200007FEF740FE06B010BD0030014000100240D4
:207E6000FFB583B0044616461D4600200290E068002804D1E068002802D1012E00D900BF11
:207E8000FF210531606888420ED1A06800280BD104215120015533460095049A11462046BA
:207EA00000F088F907B0F0BD00BF5020005D012801D10220F6E701215020015500BFFEF7CB
:207EC0000FFF07465120005D012802D00220029082E00498002801D0002E02D1012002901F
:207EE0007AE0042151200155002060650498A063A687E68700202063A086E08620646064A7
:207F00004903A068884205D12068006849108843216808602068006840210840402804D093
:207F200020680068084321680860E068002822D11DE020688068C007C00F00280AD0206825
:207F4000007BA16B0870A06B401CA063E08F401EE0870CE0FEF7C4FEC01BA84202D3681CC3
:207F6000002801D1002D02D10320029034E0E08F0028DED121E01DE020688068C007C00FF4
:207F800000280AD02068C068A16B0880A06B801CA063E08F401EE0870CE0FEF7A1FEC01B62
:207FA000A84202D3681C002801D1002D02D10320029011E0E08F0028DED13A462946204643
:207FC00001F0D2FA002801D020206065606D002801D00120029000BF01215120015500BF06
:207FE00000215020015500BF02985BE7FFB583B0044616461D4600200290E068002804D118
:20800000E068002802D1012E00D900BF00BF5020005D012802D1022007B0F0BD01215020B6
:20802000015500BFFEF75CFE074601965120005D012802D002200290B2E00498002801D054
:20804000002E02D101200290AAE00321512001550020606504982063A686E6860020A06338
:20806000A087E087606420640121C903A068884205D1206800684910084321680860206887
:20808000006840210840402804D0206800680843216808600121C902E068884232D160689D
:2080A000002802D00198012809D1206B00882168C860206B801C2063E08E401EE0861DE08D
:2080C000206880680221084002280AD1206B00882168C860206B801C2063E08E401EE08620
:2080E0000CE0FEF7FDFDC01BA84202D3681C002801D1002D02D10320029051E0E08E002811
:20810000DED131E06068002802D00198012809D1206B007821680873206B401C2063E08E62
:20812000401EE0861DE0206880680221084002280AD1206B007821680873206B401C20632D
:20814000E08E401EE0860CE0FEF7CAFDC01BA84202D3681C002801D1002D02D10320029078
:208160001EE0E08E0028DED13A462946204601F04CFA002801D020206065A068002809D128
:2081800000BF00902068C068009020688068009000BF00BF606D002801D00120029000BF9A
:2081A00001215120015500BF00215020015500BF029831E7FFB587B004461D46109E012058
:2081C000039000200290E068002804D1E068002802D1012D00D900BF00BF5020005D012857
:2081E00002D102200BB0F0BD01215020015500BFFEF776FD07465120005D04906068059007
:208200000695049801280DD0FF2105310598884205D1A068002802D10498042802D00220CF
:208220000290E9E00898002804D00998002801D0002D02D101200290DEE05120005D042842
:2082400002D0052151200155002060650998A063E587A58708982063E586A58600202064E1
:2082600060642068006840210840402804D0206800680843216808600121C902E06888423A
:208280004FD16068002802D00698012809D1206B00882168C860206B801C2063E08E401E21
:2082A000E08637E02068806802210840022811D1E08E00280ED0039801280BD1206B008833
:2082C0002168C860206B801C2063E08E401EE0860020039020688068C007C00F00280ED052
:2082E000E08F00280BD02068C068A16B0880A06B801CA063E08F401EE08701200390FEF741
:20830000EFFCC01BB04205D3701C002802D00320029071E0E08E0028C4D1E08F0028C1D1ED
:2083200050E06068002802D00698012809D1206B007821680873206B401C2063E08E401E6D
:20834000E08639E02068806802210840022811D1E08E00280ED0039801280BD1206B0078A0
:2083600021680873206B401C2063E08E401EE0860020039020688068C007C00F00280ED09E
:20838000E08F00280BD02068C068A16B0870A06B401CA063E08F401EE08701200390FEF7F0
:2083A0009FFCC01BB04202D3701C002801D1002E02D1032002901FE0E08E0028C2D1E08FAD
:2083C0000028BFD13A463146204601F01EF9002804D001200290202060650DE0A0680028AF
:2083E00009D100BF01902068C068019020688068019000BF00BF00BF01215120015500BF2C
:2084000000215020015500BF0298EBE670B504462546681E0949884201D901200CE0681E62
:20842000074948610321081F00F04AFF00200449886107200861002070BD0000FFFFFF008F
:2084400000E000E070477047FEB504462068C56920680668206887682807000F0190019866
:2084600000280ED12020284000280AD020203040002806D0206E002802D02046216E884751
:20848000FEBD019800287DD0F807C00F002804D1FF20213030400028F5D0E807C00F002895
:2084A0000BD0FF2001303040002806D0012021680862E06F01210843E0670220284000285A
:2084C0000AD0F807C00F002806D0022021680862E06F04210843E0670420284000280AD04D
:2084E000F807C00F002806D0042021680862E06F02210843E0670820284000280ED02020BF
:208500003040002803D1F807C00F002806D0082021680862E06F08210843E067E06F002887
:2085200046D020202840002809D020203040002805D0206E002802D02046216E8847E06F34
:2085400000902068806840210840402804D0082100980840002826D0204601F0FCFD206837
:20856000806840210840402819D120688068884321688860E06E00280DD02548E16E886372
:20858000E06E00E015E0FEF77BF8002810D0E06E816B88470CE02046FFF755FF08E0204655
:2085A000FFF751FF04E02046FFF74DFF0020E06766E701200005284000280CD001208005FD
:2085C0003840002807D001200005216808622046FFF738FF54E78020284000280AD0802093
:2085E0003040002806D0606E002802D02046616E884745E740202840002807D0402030407E
:20860000002803D0204601F0B8FD39E700BF37E795A0000810B50446002C01D1012010BD1E
:20862000A069002800D000E000BF606F002805D1002170200155204600F02CF82420606741
:20864000206800684008400021680860204601F0FBFD012800D1E2E7606A002802D0204675
:2086600001F08AFB206840680921C902884321684860206880682A218843216888602068E4
:2086800000680121084321680860204601F0ECFBC5E7000010B586B00446142101A8FCF714
:2086A0009AFD36492068884266D13548406B0121890308433249486300BF0846C06A01217B
:2086C00008432F49C8620846C06AC007C00F009000BF00BF032040020190022002900020C7
:2086E0000390032004900420059001A905200007FEF7F0F923482449086003204860002197
:2087000021488160C160802101610021416181612021C16100210162FEF764F8002801D015
:20872000FDF7C2FA00BF1848E066846200BF154814381649086003204860102113488160D7
:208740000021C16080210161002141618161C1610162FEF747F8002801D0FDF7A5FA00BF2B
:208760000A48A066846200BF002201211B20FEF7DFFC1B20FEF7D0FC06B010BD00380140B5
:208780000010024030000240901A0020D81A002070B504460D461646A06F202863D1002D63
:2087A00001D0002E01D1012070BD01210903A068884208D12069002805D1E807C00F002854
:2087C00001D00120F0E700BF7020005D012801D10220E9E701217020015500BF656558202E
:2087E00006530020E0672220A067E06E002820D01E48E16EC8621E48E16E08631D48E16E57
:2088000048630020E16E88632368194624313346626DE06EFEF73AF800280AD01020E067DE
:2088200000BF00217020015500BF202060670120BAE700BF00217020015500BF2068006875
:20884000FF2101310843216808602068806801210843216888602068806840210843216897
:2088600088600020A0E702209EE70000FFA0000849A10008ADA0000870477047FFB583B07F
:2088800004460D461746606F202875D1002D01D0002F02D1012007B0F0BD01210903A068C6
:2088A000884208D12069002805D1E807C00F002801D00120EFE700BF7020005D012801D139
:2088C0000220E8E701217020015500BF0020E06721206067FEF704FA0190502007535220B1
:2088E000075301210903A068884205D12069002802D10026029502E02E460020029021E0FE
:2089000006980090002280212046019B01F08AFE002801D00320BEE7002E09D10298008800
:20892000C005C00D216888620298801C029003E0307821688862761C5220005B401E81B27C
:20894000522001535220005B0028D9D106980090002240212046019B01F064FE002801D0B3
:20896000032098E72020606700BF00217020015500BF00208FE7FFE702208CE7704700BF42
:20898000FEE710B50022042105200007FEF7A1F90022082105200007FEF79BF90A2002F00F
:2089A000C9F90122042105200007FEF792F90A2002F0C0F90022042105200007FEF789F942
:2089C00010BD10B50022042105200007FEF781F90122082105200007FEF77BF90A2002F026
:2089E000A9F90122042105200007FEF772F90A2002F0A0F90022042105200007FEF769F982
:208A000010BD70B50546002400261EE00022042105200007FEF75DF90A2002F08BF9012250
:208A2000042105200007FEF754F96006040E082105200007FEF744F9002801D0601CC4B2B9
:208A4000052002F077F9701CC6B2082EDEDB002D02D1FFF7B6FF01E0FFF793FF204670BDF5
:208A600070B504460022042105200007FEF731F900252AE080202040C011002806D00122D4
:208A8000082105200007FEF724F905E00022082105200007FEF71DF96006040E0A2002F074
:208AA00049F90122042105200007FEF712F90A2002F040F90022042105200007FEF709F941
:208AC0000A2002F037F9681CC5B2082DD2DB70BD10B50122082105200007FEF7FAF80122F9
:208AE000042105200007FEF7F4F80022082105200007FEF7EEF80A2002F01CF9002204217A
:208B000005200007FEF7E5F810BD10B50022042105200007FEF7DDF8002208210520000711
:208B2000FEF7D7F80A2002F005F90122042105200007FEF7CEF80122082105200007FEF7BB
:208B4000C8F80A2002F0F6F810BD10B500240122082105200007FEF7BCF8062002F0EAF87A
:208B60000122042105200007FEF7B3F8062002F0E1F807E0601CC4B2FA2C03DDFFF7C5FF57
:208B8000012010BD082105200007FEF799F80028F0D10022042105200007FEF79AF8002009
:208BA000EFE7000038B500203D49087001F094F901F0E6F93B480068C069082108400028D9
:208BC00002D039483949C86080213948FEF778F800280BD1012251033548FEF77AF8002290
:208BE000012109033248FEF774F811E00022012149032F48FEF76DF80121C9022C48FEF7C4
:208C00005FF8002804D0012211032948FEF761F82848808C012820D100242748009072B62A
:208C200080212648FDF75CF80446002C05D0022269462248FDF746F9044662B620A001F00F
:208C400027FE00211B48818402F034FE642002F067F815481549C86000BF1648408C012878
:208C60000ED1002113484184002012494039088002F020FE642002F053F80B480B49C860B8
:208C80000C48008C01280AD100210A48018402F011FE642002F044F803480449C86038BD90
:208CA000E7000020101A00200400FA0500ED00E000040050C40D0020AAAA0000384A000870
:208CC000BDF8C8EBC9FDBCB6C4A3CABD0D0A000008B53721202000F073F80321212000F0EA
:208CE0006FF84021222000F06BF80821232000F067F8AA21302000F063F80A48008FC1B2A2
:208D0000322000F05DF80221332000F059F85F21202000F055F8684600F006F80A2002F050
:208D200009F808BD840D002010B5044621460F2000F023F8002800D110BD0120FCE770B51D
:208D400004460025FFF7C4FE3220FFF789FEFFF7FCFEE0B2FFF784FEFFF7F7FEFFF7B8FE8C
:208D60003320FFF77DFEFFF7F0FE0020FFF749FE0546FFF7CAFE284670BD70B505460C4688
:208D80002846FFF7DCFF2070012070BD70B504460D46FFF79DFE3220FFF762FEFFF7D5FEF2
:208DA000E0B2FFF75DFEFFF7D0FE2846FFF758FEFFF7CBFEFFF7A9FE0A2001F0BBFF70BDF4
:208DC00070B504460D4629462046FFF7DFFF012070BD000010B50248FEF735F810BD0000DC
:208DE00088190020F0B585B004460020039072B64F4920684018002806D14E48C06803215A
:208E000089040840039000E000BF00BF2068806802902068C068019020684569206886699C
:208E200043492068401800280DD142484038806A490508433F49403988620846806A4000D8
:208E40004008886200E000BF00BF002D01D1002E5FD0374920684018002807D13548C06821
:208E60000321890488433349C86000E000BF00BF002D1DD02068006901210843216808610A
:208E800020684561FDF72CFF074600BFFDF728FFC01B00902068006808210840082804D08E
:208EA0007D21C90000988842F0D9082021684860002E1DD02068006901210843216808615C
:208EC00020688661FDF70CFF074600BFFDF708FFC01B00902068006810210840102804D03D
:208EE0007D21C90000988842F0D91020216848600F4920684018002809D10E48C0680321A3
:208F000089048843039908430A49C86000E000BF00BF206800694008400021680861029834
:208F20002168886001982168C86062B605B0F0BD0084FFBF401002401CB500200090019016
:208F40001E481F49086000211D48C163012080071B49486000211A488160072181630121EB
:208F600001610021C160001D01774177001F8162FF21C231416200212430017204212438DF
:208F800041610021016381614163C161FDF778F9002801D0FCF788FE0A4800908013019025
:208FA00069460748FDF7E0F8002801D0FCF77CFE00210348FDF76AF81CBD00000024014081
:208FC0002C1900200200000408B500BF0A48006B01210843084908630846006BC007C00F75
:208FE000009000BF00BF002201210A20FEF7A0F80A20FEF791F808BD0010024000B587B0BD
:20900000142102A8FCF7E7F800BF6548C06A042108436349C8620846C06A0421084001904D
:2090200000BF00BF00BF5E48C06A802108435C49C8620846C06A80210840019000BF00BFF8
:2090400000BF5748C06A012108435549C8620846C06AC007C00F019000BF00BF00BF084629
:20906000C06A022108434E49C8620846C06A02210840019000BF00BF01224A4905200007C3
:20908000FDF727FE012291024748FDF722FE002246494548FDF71DFE00228121090205201D
:2090A0000007FDF716FE01200290414803900020049002A905200007FDF70CFD0220029096
:2090C000032003900020049002A905200007FDF701FD0C2002901120039000200490032004
:2090E000059002A905200007FDF7F4FC1020029001200390002004900220059002A905206F
:209100000007FDF7E7FC012002901120039000200490059002A92448FDF7DCFC022002901A
:20912000244803900120049002A91F48FDF7D2FC214802900120039000200490059002A904
:209140001948FDF7C7FC0120C0020290002003900220049002A91448FDF7BCFC91200002B3
:2091600002900120039000200490059002A905200007FDF7AFFC80200290002003900120E4
:20918000049002A90848FDF7A5FC002201210520FDF7CEFF0520FDF7BFFF07B000BD000036
:2091A000001002401C100000000400500930000000001110000021100834000010B50F48FA
:2091C0000F4908600020486000210D4881600D4941610021016241628162FDF7BFFE0028D5
:2091E00001D0FCF761FD084A511C0548FDF746FF002801D0FCF758FD10BD0000007C00403E
:2092000088190020FFFF0000FF7F000010B5124812490860FF200530486000210F488160DA
:20922000C160016141610121490281610021C1610162416281620721C162FEF793FD002896
:2092400001D0FCF731FD0548006800684021084302490968086010BD00300140B819002000
:2092600010B5134813490860E12040024860002110488160C16001610C2141610021816170
:20928000C161016200200B4948620846FFF7C2F9002801D0FCF708FDC82207490548FFF7BE
:2092A00077FA002801D0FCF7FFFC01F0FDF910BD00380140101A0020BC0C00207047000040
:2092C00010B5002819DA1A4A03071B0F083B9B089B00D2588307DC0EFF23A3409A438B0783
:2092E0001B0E8407E40EA3401A43114B0407240F083CA408A4001A5118E00E4A03231B025C
:20930000D21883089B00D2588307DC0EFF23A3409A438B071B0E8407E40EA3401A43054BF5
:20932000032424021B198408A4001A5110BD00001CED00E000E100E070470000F0B585B009
:209340004D484E49086002F055FAFF200A304C4948800846C08E4B4908704948C08F4A4967
:2093600008704748808F494908704548807A48490870434880884749086041490889FCF7A4
:20938000CFF906460022444BFCF7C4F804460022424BFCF727F90191009001F05DFC03914D
:2093A0000290FCF7DFF93E4908803549C8883C490988FBF7B3FE3B490880314988883949A2
:2093C0000988FBF7ABFE36480088414388B236490880084600880A30FCF77CF93349029010
:2093E000FBF76AFF0390FCF7DBF90646304A314BFCF7F8F80446FCF7B5F92F49088008465A
:2094000000882E4908801E49C888FCF76EF927490290FBF751FF0390FCF7C2F90446244A77
:20942000244BFCF7DFF80646FCF79CF9244908801348C1887D20C000FBF770FE21490880D7
:209440001D48028820492148FDF718FE002801D0FCF72AFC0F4801681DA001F019FA08485E
:20946000C1881FA001F014FA0548018921A001F00FFA05B0F0BD0000B5A600084800002026
:20948000840D0020010000203801002039010020270100201C01002000001040000008402A
:2094A0002C0100202E0100202801002000007A44F853E3A59B843E403401002030010020F3
:2094C00032010020360100204781000088190020B1EAC7A949443A202564202E0D0A000079
:2094E000CDA8D1B6BCE4B8F43A202564206D732E0D0A0000B5A5B4CECDA8D1B6BBF9D5BEDD
:20950000CAFDC1BF3A202564B8F62E0D0A00000000B585B014216846FBF75DFE00220121D0
:20952000C9031048FDF7D5FB0120C00300900120019000200290039069460A48FDF7CAFA1F
:209540000120C00300900320019000200290039069460448FDF7BEFA022001F0E1FB05B053
:2095600000BD000000040050F8B504460E461546FF210531606888420ED10121C903A06877
:20958000884203D04911A068884205D1206800684021884321680860FF2105316068884237
:2095A00022D101218902A06888420ED03346002280212046009500F055F8002823D0606DFF
:2095C0002021084360650320F8BD3346002201212046009500F046F8002814D0606D202162
:2095E000084360650320EFE73346002201212046009500F037F8002805D0606D2021084335
:2096000060650320E0E70020DEE7F8B504460E461546FF210531606888420ED133460022AE
:2096200080212046009500F01DF8002818D0606D2021084360650320F8BD5120005D052888
:209640000ED13346002201212046009500F00AF8002805D0606D2021084360650320EBE771
:209660000020E9E7F8B504460E4617461D4641E0681C00283ED0FDF733FB0699401AA8420F
:2096800001D2002D36D120684068E021884321684860FF210531606888420ED10121C903E1
:2096A000A068884203D04911A068884205D120680068402188432168086001214903A06A7E
:2096C00088420DD100BF20680068884321680860206800680121490308432168086000BF1E
:2096E00001215120015500BF00215020015500BF0320F8BD206880683040B04201D101207F
:2097000000E00020B842B3D10020F2E77047000038B504460D460020009055201B49087090
:20972000AA20487003208870601DC870032008710846457184716800154A8118224613481F
:20974000C01DFBF72FFD002008E0811C0F4A525C6946098851188AB20092401C611D884247
:20976000F3DB0A48801CFCF7EDF90090E01D074941186846007808706846407848702146FB
:209780000931024800F012FD38BD0000C7180020840D002001460020054A126890B2054AE0
:2097A000104002460A431046014A10607047000000300140C7FF000010B5FDF797FA10BDAE
:2097C00000B599B034210CA8FBF705FD142107A8FBF701FD1C216846FBF7FDFC2448006810
:2097E0000321C90288430121C902401820490860FDF7B0FC1F4800690321C90288431D4909
:20980000086106200C9088150E9001200F9010201090022015900021169141041791410590
:2098200018910CA8FDF78CFF002801D0FCF73CFA0F20079003200890002009900A900B90BB
:20984000012107A8FDF7E6FD002801D0FCF72CFA8120009000200290032080040690684680
:20986000FDF7C2FC002801D0FCF71EFA19B000BD007000404010024015480068FF21013153
:209880000843134908600846C068124908401049C86008460068104908400D4908600846BC
:2098A000806840084000886008460068012189048843074908600846C068FD2109048843FC
:2098C0000349C860002008610448054988607047001002400C40FF88F6FFF6FE00500008EC
:2098E00000ED00E0F0B58DB000200A9001F0E4FC0B9002E001F0E0FC0B90F4490B9888429F
:20990000F8D10020F2490880962001F030FD4B20C00001F049FD0020EE490870EE480078E8
:20992000EE49C873EE4801780068401CEC4A1060C8B2EA4948740025BFE1E8488573002224
:209940000146142001F016FE0021142001F026FE022001F067FDE3490870E348076805E083
:2099600000210F2001F08EFCE049086000210F2001F088FCDD490860DD4908400028EFD0E3
:20998000DA48006801218903084000287DD08122D20100210F2001F0A6FD0021102001F036
:2099A00071FC4006400ED34908600846008881B20022D14801F0B6FCCF480078CF49097813
:2099C00088427DD1CC48407A0228FAD10422CC49C948401DFBF70AFC0028F2D101F03BFEF6
:2099E000C84A03C201F020FEC74A03C20A9800282AD1C648C089002826D001200A90C449A9
:209A0000BD48C0890880C348BB49098A01800088FF30C330BF49088008460088BE4988426C
:209A200012DDBC480088401ABA490880B8480088401CB749088008460088B7490B3188427E
:209A400002DB0020B2490880B449AB4842890A80808948800422A849491CB148FBF7A2FB6C
:209A6000A548418A08916846008C042813DDA748C0886946098C88420DD06846008CA349F7
:209A8000C88001F017FF642000E00CE101F048F9A448A549C8609C4803684068A34A0021ED
:209AA0009A1848410106140A0C43204601F057FC6108490000200A0E000210430B0200E021
:209AC000EDE0002211469A18484199490A6048608C480CC89248093001F08CFD8A480CC836
:209AE0008F480D3001F086FD91480CC88C48113001F080FD00228A49491E182001F03AFDF2
:209B00000021182001F04AFD012001F08BFC754908707F4800887D21C90048437D4909884D
:209B20004018844908608448FDF7A4FA86B2774AD2887D23DB005A4311467E4A12687F4B6C
:209B4000D01AFBF7EBFA7E4800887D22D20050436E4AD2887D23DB005A438018401A794914
:209B6000401A7949086073490968784A881A002801DB014600E041427D22D200914205DAFF
:209B8000714800686D4940186F4908606E4800687D210901884208DA5C48C0884910484334
:209BA0006949096840186849086067480068FBF7A3FD674A674B01910090FBF713FD05914B
:209BC00004903046FBF7ACFD03910290059B049AFBF7EEFB07910690FBF7C4FD5E49088091
:209BE000084600885D49884204DD5B480088401A59490880584800884F4909684861354838
:209C00000078401C334908703B48427808A90A71807848713D48C08B00282AD101205049B5
:209C200088701120C8702E4800780871084634490A784271497881712F494A78C27189783B
:209C40000172042235490930FBF7ACFA454800784349487344480078887311214048801C7B
:209C6000FBF770FF414908803D480A78C274497801751C480078002808D100BF00210F2011
:209C800001F000FB802108400028F7D0802200210F2001F028FC0020354908700BE00120D7
:209CA0003349087007E0334A00210F2001F01BFC01202F490870681CC5B214480089A84219
:209CC00000DD3AE601F0CCF90DB0F0BD3001CADEE8000020EB00002042010020841500205F
:209CE0006C000020EA000020FC0000207400002000D0272404010020D4150020270100208D
:209D00001C0100207800002080000020840D002024010020F8000020E7030000F0000020C6
:209D2000A71500200400FA0500ED00E0000052038800002000010020881900201027000061
:209D4000280100201E1400000C010020B0E20D00F853E3A59B843E40300100204781000033
:209D60004A180020E4000020E5000020F4000020B800002000902724818CC907C90F0029B3
:209D800008D001684968012252049143826A1143026851600222416A1140022907D101689D
:209DA0004968D2039143C26A1143026851600422416A1140042907D1016849681204914383
:209DC000026B1143026851600822416A1140082907D10168496812039143426B114302680A
:209DE00051601022416A1140102907D10168896812029143826B1143026891602022416AA8
:209E00001140202907D10168896812029143C26B1143026891604022416A1140402915D105
:209E20000168496892039143026C11430268516001221205016C914208D101684968032230
:209E400052059143426C1143026851608022416A1140802907D10168496812039143826CAA
:209E6000114302685160704738B504460020E067FCF736FF0546206800680821084008281A
:209E80000BD114482B46002289040090204600F0C9FB002801D0032038BD2068006804219A
:209EA000084004280BD10B482B46002209050090204600F0B7FB002801D00320ECE7202097
:209EC0006067A06700BF00217020015500BF0020E2E70000FFFFFF0170B50025C8242048AA
:209EE0000078002800D070BD1E480078002800D0F9E701201B4908701B48406B002801D10A
:209F00000870F0E71848406BC8210D1A1CE01749174A1268885C1749096888471648008836
:209F20003C2148431549088011480068401C1049086008460068C82801DB002008600A4819
:209F4000406BC8210D1A641E09480068A84201D0002CDCDC00200349087000BFC3E700001F
:209F6000420000204400002000000240BC0C00203800002048000020360100204001002079
:209F800010B53A480078002803D139480078002800D010BD0120364908703648C0698021E8
:209FA0000840002802D132490870F2E7324900200856324900228A56904215D12D48C069C6
:209FC0004021084000280BD02D480078002807D000202B4908702B480088401C294908808C
:209FE000002023490870D4E725480078002805D10120234908700A2000F09CFE1F4900207E
:20A000000856CC21484320494018001D1F490968405C184988621D480068401C1B490860D7
:20A02000164900200856CC2148431749085817490968884214DC0020144908600F480078CC
:20A04000401C40B20D490870084600780E2801D1002008700E480078401C40B20C49087095
:20A0600000200349087000BF93E700004200002043000020003801403500002034000020DC
:20A08000450000205200002094010020580000203600002070B50546AC6A00215A200153F1
:20A0A000522001532046FEF7CEF970BDF8B50546AC6A666FA76F2068806880210840802891
:20A0C00007D1212E05D1002152200153204600F064F82068806840210840402807D1222F40
:20A0E00005D100215A200153204600F034F8E06F10210843E0672046FEF7A5F9F8BD70B534
:20A100000546AC6A2868006820210840002817D100215A20015320680068FF210131884351
:20A12000216808602068806840084000216888602068806840218843216888602020A06771
:20A140002046FEF799FB70BD70B50446A56A2846FEF793FB70BD01680968FF222132914325
:20A16000026811600168896849084900026891602021816700210166704710B504462068B6
:20A180000068402188432168086020206067002060662046FEF7F2FB10BD01680968C0227C
:20A1A00091430268116020214167704770B505460C4620480078002803D11F4800780028AB
:20A1C00000D070BD01201B490870C82C04DC1B4800214156002903DC002016490870F0E7C0
:20A1E000174900200856CC21484316490C50144A00215156CC225143124A8918081D22461C
:20A200002946FAF7CFFF0E480078401C40B20C490870084600780E2801D100200870074872
:20A220000078401E40B20549087000200149087000BFC6E742000020430000203600002027
:20A240003500002094010020F0B587B00446102004900025002003900026E749206888428A
:20A2600000D100E000BF2169A068084361690843E1690843074620680068E04908403843BE
:20A280002168086020684068032109038843E168084321684860A769D7492068884201D08A
:20A2A000206A0743206880680B210902884338432168886000BFD249206888421CD1D1483A
:20A2C000C0688007800F002806D001280AD0022805D003280CD108E0012004900BE002208E
:20A2E000049008E00420049005E00820049002E01020049000BF46E0C349206888421CD1B3
:20A30000C048C0680C210840002806D004280AD0082805D00C280CD108E0002004900BE0F7
:20A320000220049008E00420049005E00820049002E01020049000BF25E0AF492068884272
:20A340001FD1B048C068032189020840002808D001218902401A0AD0401A05D0401A0CD1AF
:20A3600008E0002004900BE00220049008E00420049005E00820049002E01020049000BFFA
:20A3800001E01020049000BF9B492068884256D1049804281AD004DC002807D002281CD154
:20A3A00008E0082816D0102817D117E0FDF73CF9064616E0934840380068102108400009E0
:20A3C000002801D0914E00E0914E0AE0FDF750F9064606E00126F60303E000BF0120039017
:20A3E00000BF00BF002E0AD0606841004018B04203D860680003B04202D201200390F4E090
:20A40000606802903046FF21013100F068FA6268520800238018594101910090029AFAF7A0
:20A4200091FE054603200002854205D37948854202D82068C560D8E001200390D5E001212C
:20A44000C903E06988426FD1049804283CD006DC002809D0012813D002284AD11CE00828A9
:20A460003ED0102845D145E0FDF7DEF8400061684908401802906168FAF73AFE85B23CE008
:20A48000FDF7E4F8400061684908401802906168FAF72EFE85B230E05A48403800681021C8
:20A4A00008400009002807D061684A085A4BD018FAF71EFE85B206E061684A08574BD018D5
:20A4C000FAF716FE85B218E0FDF7D2F8400061684908401802906168FAF70AFE85B20CE061
:20A4E00061684A0801231B04D018FAF701FE85B203E000BF0120039000BF00BF102D0FD3FC
:20A50000474885420CD846480F38284005902807400F05990843059005982168C86064E0A1
:20A520000120039061E0FFE7049804283AD006DC002809D0012812D0022847D11AE0082814
:20A540003BD0102842D142E0FDF76EF861684908401802906168FAF7CBFD85B23AE0FDF75E
:20A5600075F861684908401802906168FAF7C0FD85B22FE0234840380068102108400009E0
:20A58000002807D061684A08204BD018FAF7B0FD85B206E061684A081D4BD018FAF7A8FD92
:20A5A00085B217E0FDF764F861684908401802906168FAF79DFD85B20CE061684A08012363
:20A5C000DB03D018FAF794FD85B203E000BF0120039000BF00BF102D05D31148854202D819
:20A5E0002068C56001E001200390002020666066039807B0F0BD000000480040F369FFEFDC
:20A6000000380140401002400044004000093D000024F400FFFF0F0000127A000048E80183
:20A62000FFFF0000FFB581B004460D4617460A9E22E0701C00281FD0FCF752FB0499401AB9
:20A64000B04201D8002E17D120680068FF21A13188432168086020688068400840002168FA
:20A66000886020206067A06700BF00217020015500BF032005B0F0BD2068C0692840A842D7
:20A6800001D1012000E00020B842D2D00020F1E710B510200349096808620248FDF7D4FE07
:20A6A00010BD0000101A00200D200149087070473600002070B5044600256A480078082899
:20A6C00065D100BF002004E06749095C49198DB2401C66490978491F8142F5DC644800781F
:20A6E000281885B261480078281885B261480078281885B260480078281885B25F480078FD
:20A70000281885B26019C007C00F002835D058480078012827D002282DD15949554A12785B
:20A72000881855490A785049FAF73CFD01F0C2F8642000F0F5FA00BF00BF00BF00BF00BFCD
:20A74000BFF34F8F00BF00BF00BF4E484E49C86000BF00BF00BFBFF34F8F00BF00BF00BFCD
:20A7600000BF00BFFDE743480078411042480078FEF7CEFF00E000BF00BF002039490870E7
:20A780003C490870394908704049087068E035480078072812D134483C49097844543B48D5
:20A7A0000078401C3949087030480078401F0978884255D108202B49087051E029480078DD
:20A7C000062805D12C48047007202649087047E024480078052805D12648047006202149FF
:20A7E00008703DE01F480078042805D12048047005201C49087033E01A480078032808D114
:20A800001A48047000201B49087004201549087026E014480078002805D1552C03D101201E
:20A82000104908701CE00F480078012805D1AA2C03D102200B49087012E00A4800780228FF
:20A8400007D1032C05D10320064908700B48047006E0002003490870064908700349087015
:20A8600070BD000012010020631800201401002017010020150100201301002016010020CF
:20A88000840D00200400FA0500ED00E0180100200FB410B503A9044B044A029800F034F976
:20A8A00010BC08BC04B0184711B60008540100202021020C01D010211046020A01D01046D7
:20A8C0000839020901D01046091F820801D01046891E420801D0881E7047081A7047F8B587
:20A8E00082B28BB2040C0D0C10465843002126465E43370C36048019794116466E43370C7F
:20A9000036048019794126466E438919F8BD30B47446641E2578641CAB4204D3635D5B001A
:20A92000E31830BC18471D46F8E702E008C8121F08C1002AFAD170477047002001E001C1BD
:20A94000121F002AFBD1704708B5002100916B46012202212C2000F0DBFD022100916B463A
:20A9600001222C2000F0D4FD08BD000038B504466D2000906B46012208492E2000F0C8FD66
:20A98000002C05D0064A07492E2000F09BFD04E0054A04492E2000F095FD38BD06080000ED
:20A9A00007060000061800000716000038B504466B4602220021362000F084FC2300FFF743
:20A9C000A6FF0E11081A54545454233154543D444B540021684601704078FE210840694617
:20A9E000487043E069460878FC21084001210843694608703AE069460878FC210840022183
:20AA000008436946087031E068460078B32108404821014368460170407880210843694652
:20AA2000487023E068460178B32001406846017040784106490E6846417017E069464878E6
:20AA4000022108436946487010E069464878FD2108406946487009E069460878CF210840A5
:20AA6000202108436946087000E000BF00BF6B4601220021362000F04BFD00AB0133012240
:20AA80001146362000F044FD38BD08B5032168464170012101706B4602220021362000F0D4
:20AAA00037FD0122D20306212D2000F00BFD012000F036F90120FFF779FF08BD38B5044633
:20AAC0002004010E6846417004706B46022204212D2000F01DFD0321684601706B46012208
:20AAE00006212D2000F014FD0021684601706B46012206212D2000F00BFD0A212D2000F0F9
:20AB0000C1FB0546284638BDFFB58DB00446002506E025280AD0109A0F999047641C6D1C2C
:20AB200020780028F5D1284611B0F0BD00270121484A009700E00743641C23780846203B53
:20AB400098401042F7D120782E2817D1042007436078641C2A280CD10E98641C02C80091B7
:20AB60000E900BE000990A22514330394018641C00902078014630390929F3D9207800281C
:20AB8000D1D0642808D0692806D075281ED0109A0F9990476D1C5BE00A200E99019001C9A5
:20ABA0000E91002802DA40422D2102E0390504D52B216A461172012103E0F90704D0202190
:20ABC000F7E70BAE0B910DE00021FAE70A200E99019001C90E91F7E70199FAF789FA30313B
:20ABE000761E31700028F7D103A8801B20300190780701D5009801E0012000900199884226
:20AC000001DD401A00E000200027009006E002A8109AC05D0F9990476D1C7F1C0B988742DF
:20AC2000F5DB04E0109A30200F9990476D1C0099481E00900029F5DC05E03078109A761C0C
:20AC40000F9990476D1C0199481E01900029F4DC641C65E709280100F8B54A002B4B520D98
:20AC6000D6182B4A0C460546142E2BDA002E12DA284BFAF79DFB00221346FAF7A5FD40D257
:20AC8000002C03DA0124E40700253AE02046284337D0214C14E0214F0B46F7403B402B4342
:20ACA00031D01C4BFAF784FB00221346FAF78CFD27D2002C03DD01200005F0400419BC4350
:20ACC00000251EE0332E1EDC33460027143BFF43DF40384217D00F4BFAF714FC002213466F
:20ACE000FAF772FD0DD2002C0ADD142E0CD03420811B012088404019A84200D2641C05462B
:20AD0000BD4321462846F8BD641CF9E701FCFFFF9C7500883CE4377E0000F03FFFFF0F00A4
:20AD200070B504467D20C00060430546284600F001F870BD002100BF40E000BF00BF00BF98
:20AD400000BF00BF00BF00BF00BF00BF00BF00BF00BF00BF00BF00BF00BF00BF00BF00BF03
:20AD600000BF00BF00BF00BF00BF00BF00BF00BF00BF00BF00BF00BF00BF00BF00BF00BFE3
:20AD800000BF00BF00BF00BF00BF00BF00BF00BF00BF00BF00BF00BF00BF00BF00BF00BFC3
:20ADA00000BF00BF00BF00BF00BF00BF00BF00BF00BF00BF00BF00BF00BF491C8142BCD329
:20ADC00070470000F0B585B004460020049003902578607940008A49085A02906078401E9E
:20ADE0008849C6B20863042D01D0072D01D1012000E000200190207882490873E079002886
:20AE00000AD1084680690121890508437D4988610298C010029006E07A4880690121890539
:20AE2000884378498861207A7649487308468069217A090403221204114008437149886130
:20AE4000084600218269042000F04DFB6E492E20029A00F037FB3046FFF788FD6B48405D38
:20AE6000810040186A494318052207212B2000F04FFB684901980B1801220B21282000F023
:20AE800047FB6248405D800063490A580C21282000F029FBE079800060494018A1794900D5
:20AEA000425A0221272000F00DFB70005C490A5A0421272000F006FBE079002805D16422E1
:20AEC0000621272000F0FEFA1EE0A07804280DD11020009010220621272000F0F3FA6B460E
:20AEE00001222621272000F013FB0DE02820009020220621272000F0E5FA6B460122262144
:20AF0000272000F005FB00BF300146494018E178890042580821272000F0E5FAA17A627A71
:20AF200008021043002803D13F496172090AA172A17A637A0802184302462021272000F01A
:20AF4000C1FA3A480C210268232000F0CCFA71003648001D425A0421232000F0B3FAA0795E
:20AF600000280BD0E0793249431801220021212000F0CEFA03200490012003902807000FB9
:20AF80002901F02211400843617889040322920411400843049909059200114008430399A7
:20AFA00049040122520411400843217989051F229205114008436179C906C90EC9060843F9
:20AFC00007463A4600211F2000F08DFAA0786178084300040B49086108460069E179490373
:20AFE0000122D2031143084306490861084600210269082000F077FA002005B0F0BD00001D
:20B000008CB90008580100200428000034B9000802000020200000203CB900085CB90008CD
:20B0200068B900086CB900084110000054B900082200002038B504460D460848808B0443E6
:20B04000224600212C2000F03DFA00956B46012206212C2000F05CFA38BD00005801002064
:20B0600010B5FFF771FC10BD70B505460421362000F008F90446002D03D00120C00204438B
:20B0800004E00121C90220468843044622460421362000F028FA70BDF0B585B006460420F8
:20B0A00002900027002001906649487508630021644820304171017300206249888348638B
:20B0C000886300F0F9F85F49086003E000F0F4F85C4908605B4800685B498842F6D1002068
:20B0E000FFF764FC59480078432802DD43205749087056480078002802DA002053490870CE
:20B1000052480078242804DD504800780446243C0DE006214D480078FAF700F80621081AE3
:20B1200045014A480078F9F7F9FF2C460C43200621040843210208432043039000211E20BD
:20B14000039A00F0D0F902AB01220021242000F0DFF91E20FFF7B2FC87B2381239498873BA
:20B160000420FFF7ABFC01900198C0B200280FD0022000906B46012212212D2000F0C8F9B4
:20B180003048808B0121090308432E49888300BF00F092F82B4908600620FFF78FFC294903
:20B1A00048600720FFF78AFC26498860F806C00E08750846007D002801D1102008752149C8
:20B1C000087D00F0FDF9F007C00F002809D0FFF75CFC1C48808B0121C902084319498883DB
:20B1E0000CE00521362000F035F80546184805402A460521362000F065F900BF0120FFF7CA
:20B20000D5FB0021042000F03DF80E4988610021262000F037F80546052080030543800073
:20B2200005432A460021262000F05DF900222621362000F047F900F03FF8024908600020C0
:20B2400005B0F0BD580100203001CADE01000020FFFD0000F8B504460D46094FA9B2A0B2CE
:20B260006B46022200F02EF80646002E06D168464078010268460078081887B23846F8BD77
:20B28000FFFF0000FEB505460E460027FF43B1B2A8B201AB042200F015F800900098002819
:20B2A00008D1032404E0380201A9095D4718641E002CF8DA3846FEBD10B500210846FFF71E
:20B2C000E1FF10BDFFB581B006460C4617460025002C04D129466D1C684646541AE0402021
:20B2E0003043C2B229466D1C684642547F2C04DC28466D1C69460C540CE0E0B28021084330
:20B3000029466D1C6A4650546004020E28466D1C69460A54A8B23A466946049B00F0AAFAAD
:20B3200005B0F0BD70B504460D46164623462A4631461120FFF7C6FF70BD10B504462346AC
:20B34000052200211520FFF7BDFF10BD10B504462346052200211720FFF7B4FF10BD10B5BF
:20B360000446224601210A2000F0BDF810BD70B5054600211A20FFF785FF0446240D240574
:20B380002803000B0443224600211A2000F0ABF870BD000010B50446224602492E2000F0AD
:20B3A00091F810BD0418000038B504466B46012203210420FFF786FF002C16DD22460021A5
:20B3C0000C2000F07FF8694608781021084300900F488069090608430D4988616B460122F2
:20B3E0000321042000F094F810E06946087810218843009006488069090688430449886197
:20B400006B4601220321042000F082F838BD00005801002010B5044622460021182000F078
:20B4200051F810BDF8B5044600250020009000260220204000280AD0802000906B4601227C
:20B4400000210D2000F064F801211D480173E007C00F002826D06946087806210843009052
:20B460006B46012200210D2000F052F803210F20FFF7F0FE06468120C0003040002801D122
:20B4800000251AE0402000906B46012200210D2000F03EF80020FFF7E7FD00210848017376
:20B4A0004D1E0AE0694608780221084300906B46012200210D2000F02BF82846F8BD0000B2
:20B4C00078010020F8B505460E4614466846047021124170B1B2A8B26B46022200F018F895
:20B4E00007463846F8BDFEB506460F461446002503E069464C55240A6D1C042DF9DBB9B29F
:20B50000B0B26B46042200F003F801900198FEBDFFB581B006460C4617460025002C07D119
:20B5200080203043C2B229466D1C6846425419E0C0203043C2B228466D1C69460A547F2CD9
:20B5400003DC28466D1C0C540CE0E0B28021084329466D1C6A4650546004020E28466D1C94
:20B5600069460A54A8B23A466946049B00F0BCF905B0F0BD70B504460E461546281901210E
:20B580008902884202DD0020C04370BDA21E334629460920FFF7BCFF0020F6E770B5044639
:20B5A0000D46064800692043A90508430646324600210820FFF797FF002070BD58010020C6
:20B5C00038B504466B4601220E212B20FFF77AFE68460078410949010091E106C90E6846C1
:20B5E0000078014300916B4601220E212B20FFF78FFF38BD70B50146002006E00A541E0643
:20B60000140A34431B0A2246401C0428F6DB70BD13B50C4601231A4669460248FDF72EF9D0
:20B6200000981CBD101A00207CB500210C460D466846FFF782FE042608E0220E2802104375
:20B64000240205466846805D0443761E002EF4DA204629467CBD7CB500210C460D46684664
:20B66000FFF774FE042608E0220E28021043240205466846805D0443761E002EF4DA20466A
:20B6800029467CBDFBF73AFBFEF79AF8FDF7B6FCFDF794FDFDF7E4FDFDF7B8FDFDF74CFC6F
:20B6A000FDF792FCFDF74AFEFDF712FBFAF7BCFAFAF77CFA0721FF204130FFF7BBFCFFF762
:20B6C000CFFC0120284908800122010305200007FBF7FFFA46E025480078002840D0FEF70F
:20B6E0006FF8002021490870FAF734FC20490870084600780F280FDD0122D10305200007D3
:20B70000FBF7E7FAFEF7EEF800220121C90305200007FBF7DEFA0BE0012208211548FBF7EF
:20B72000D8FAFEF7DFF8002208211248FBF7D1FAFDF738FA0C480088002804DD0A48008824
:20B74000401E094908800C48007800280AD106480088002806D101210846FBF721FD01E0AC
:20B76000FDF720FAB7E7000040010020E600002042010020000400504500002000B585B0B0
:20B780001748FBF746FB14216846F9F724FD154800900320019000200290694605200007F5
:20B7A000FBF798F969461048FBF794F969460F48FBF790F901210846FBF7F2FCFF2001305F
:20B7C000FBF7C0FC0A48006804210843084908608815FBF7C9FCFBF7CFFC05B000BD000055
:20B7E00088190020FFFF000000040050000800500070004010B50122D2021B491B48FAF7BA
:20B800008AFA194800881A4988422CD0084616490880042088807D20C000C88001200881E2
:20B82000002048811E20C04388810120C88100200884088248828882C8820883888343201E
:20B84000C886012008877820488701208887C887002105484030018441848184002002496C
:20B86000C88300F027F810BD840D002000F00008AA550000F8B504460F4615461E460020CE
:20B88000009010200521090788620A23224639460748FCF7ABFBAAB20A2331460448FCF78D
:20B8A000DFFA10200521090788610020F8BD0000B819002010B5002472B60121C90208484C
:20B8C000FAF70EFA0446002C06D00122D20205490348FAF7F7FA044662B6204610BD00001C
:20B8E00000F00008840D0020F8B504460F4615461E460020009010200521090788620A2367
:20B90000224639460948FCF771FB09490870AAB20A2331460548FCF769FB0549087010202C
:20B920000521090788610020F8BD0000B8190020250000200000010203040005405C000032
:20B94000A05C0400C06C0800805C0400E03F1E00E07D1E0007A9022570889B880A00160009
:20B96000010006000100020087008D002D001A3152001A339A001A351D011A376B003B3163
:20B98000BE003B335E013B3596023B37000099599959EB518F421E45142E0080EB51F52833
:20B9A0003333E13A703DE13AC235852BC2353333C235C235AE47E13A5138A3305138000057
:20B9C00000000000000001020304060708090000000001020304030406080C10182030009C
:20B9E00000BA000800000020580100001C5A000838BA000858010020E01D00003AA9000833
:20BA000021130704380D091E080540082609104008560A131D043B08BE0596D8BC40100883
:18BA2000042FC8420114020214150909010202AD81092EE7B152200009
:00000001FF
